:1000000000802020650600006106000061060000F7
:1000100000000000000000000000000000000000E0
:100020000000000000000000000000006106000069
:10003000000000000000000061060000F51800004C
:100040006106000061060000610600006106000014
:100050006106000061060000610600006106000004
:1000600000000000610600006106000000000000C2
:10007000000000006106000061060000610600004B
:1000800061060000610600006106000061060000D4
:100090006106000061060000000000000000000092
:1000A0006106000061060000000000000000000082
:1000B000610600000000000061060000610600000B
:1000C000002243088B4274D303098B425FD3030A97
:1000D0008B4244D3030B8B4228D3030C8B420DD3AA
:1000E000FF22090212BA030C8B4202D31212090238
:1000F00065D0030B8B4219D300E0090AC30B8B4276
:1001000001D3CB03C01A5241830B8B4201D38B0323
:10011000C01A5241430B8B4201D34B03C01A5241C8
:10012000030B8B4201D30B03C01A5241C30A8B420B
:1001300001D3CB02C01A5241830A8B4201D38B02F6
:10014000C01A5241430A8B4201D34B02C01A52419A
:10015000030A8B4201D30B02C01A5241CDD2C3090C
:100160008B4201D3CB01C01A524183098B4201D388
:100170008B01C01A524143098B4201D34B01C01A73
:10018000524103098B4201D30B01C01A5241C308EB
:100190008B4201D3CB00C01A524183088B4201D35A
:1001A0008B00C01A524143088B4201D34B00C01A46
:1001B0005241411A00D20146524110467047FFE7B2
:1001C00001B5002000F006F802BDC0460029F7D0B6
:1001D00076E770477047C046024670B50A439207FB
:1001E0002AD11E4DEE0104C808C9541B9443344063
:1001F00017D0D0B2D9B2401A2106014310D190B223
:1002000099B2401A210401430AD110021902000ACE
:10021000090A401A2102014302D1100E190E401A98
:1002200070BD9A42DFD010BA19BA884201D90120B4
:1002300070BD0020C04370BD02780B7801300131E1
:10024000002A09D09A4207D102780B780130013197
:10025000002A01D09A42EFD0D01A70BD01010101ED
:1002600003460B437FD4002243088B4274D3030917
:100270008B425FD3030A8B4244D3030B8B4228D3B8
:10028000030C8B420DD3FF22090212BA030C8B42DE
:1002900002D31212090265D0030B8B4219D300E07E
:1002A000090AC30B8B4201D3CB03C01A5241830B03
:1002B0008B4201D38B03C01A5241430B8B4201D3B3
:1002C0004B03C01A5241030B8B4201D30B03C01ADC
:1002D0005241C30A8B4201D3CB02C01A5241830A56
:1002E0008B4201D38B02C01A5241430A8B4201D385
:1002F0004B02C01A5241030A8B4201D30B02C01AAF
:100300005241CDD2C3098B4201D3CB01C01A524115
:1003100083098B4201D38B01C01A524143098B429E
:1003200001D34B01C01A524103098B4201D30B0187
:10033000C01A5241C3088B4201D3CB00C01A5241AC
:1003400083088B4201D38B00C01A524143088B4271
:1003500001D34B00C01A5241411A00D2014652410A
:10036000104670475DE0CA0F00D04942031000D329
:100370004042534000229C4603098B422DD3030A7E
:100380008B4212D3FC22890112BA030A8B420CD38E
:10039000890192118B4208D3890192118B4204D3B7
:1003A00089013AD0921100E08909C3098B4201D337
:1003B000CB01C01A524183098B4201D38B01C01A71
:1003C000524143098B4201D34B01C01A52410309E8
:1003D0008B4201D30B01C01A5241C3088B4201D397
:1003E000CB00C01A524183088B4201D38B00C01A44
:1003F0005241D9D243088B4201D34B00C01A52411B
:10040000411A00D20146634652415B10104601D3A7
:100410004042002B00D54942704763465B1000D331
:10042000404201B50020FFF7D5FE02BD0029F8D0FB
:1004300016E77047002B11D1002A0FD1002900D1F7
:10044000002802D00021C943081C07B4024802A1B9
:100450004018029003BDC0467DFDFFFF03B468460F
:1004600001B5029800F006F8019B9E4602B00CBC54
:100470007047C046F0B557464E464546DE46E0B5A5
:1004800004000D009246994683B08B4230D82DD09F
:100490004946504600F0BAF829000600200000F056
:1004A000B5F8331A9846203B9B4633D45A465346F8
:1004B000934042461F00534693401E00AF423AD835
:1004C000AF4200D178E05B46A41BBD41002B00DAAF
:1004D00075E0002200230092019301235A469340C5
:1004E0000193012342469340009328E08242CFD9F2
:1004F00000220023009201930C9B002B01D01C6072
:100500005D600098019903B03CBC90469946A246B4
:10051000AB46F0BD424620239B1A5246DA40414684
:1005200013004A468A40170042461F4353469340F1
:100530001E00AF42C4D9002200230092019343461B
:10054000002BD9D0FB0772081A4346467B080EE001
:10055000AB4201D1A2420CD8A41A9D41012024191A
:100560006D410021013E24184D41002E06D0AB42C2
:10057000EED9013E24196D41002EF8D10098019961
:100580005B4600196941002B24DB2B005A46444688
:10059000D3402A00E2401C005B461500002B2ADBFA
:1005A00026009E40330026004746BE403200801A97
:1005B0009941009001919FE7A342BCD883E742464E
:1005C000202300219B1A0022009101920122DA408F
:1005D000019286E7424620239B1A2A0046469A400B
:1005E0002300F340444613432A00E2401C005B46CC
:1005F0001500002BD4DA42462F0020232600974016
:100600009B1ADE403B003343CDE7C04610B50029BE
:1006100003D100F007F8203002E0081C00F002F8D7
:1006200010BDC0461C2101231B04984201D3000CBD
:1006300010391B0A984201D3000A08391B09984255
:1006400001D30009043902A2105C40187047C0466B
:10065000040302020101010100000000000000008B
:10066000FEE7000010B50F4B0F4A10498B4202D233
:1006700002CA02C3F9E70E4B0E4A0F498B4202D25F
:1006800002CA02C3F9E70D4B01E0002204C30C4A81
:100690009342FAD302F0B6FF00F015F8FFF7E0FF3F
:1006A00010BDC0464000202090670000B80C2020FC
:1006B000000020208861000040002020B80C20208D
:1006C00018322020704710B501F03AF900F054F8C4
:1006D000002010BD10B5074C074B236000F080FAD6
:1006E0006060200000F062F800F04CF8034800F071
:1006F0007BFA10BDB80C20204000202028012020CB
:1007000010B501F0FFF8040006E000F067F8194B9F
:100710001860012001F0FCF8164B1B68002B06D175
:1007200001F0F0F8001BC8235B009842EDD3114B99
:100730001B68012B09D000F0D7FC002812D16420DF
:1007400001F0E6F801F018F910BD792000F09EFBE9
:10075000C046002400E0002400F05EF80134642C60
:10076000F9DCF9E7642001F0D3F88020000200F002
:100770006FFCE4E7C00C202010B5FFF7ABFFFFF7DC
:10078000BFFF10BD10B50024064B1B68A34200D864
:1007900010BDE300044A9B581B68002B00D098470B
:1007A0000134F1E7C40C2020C80C202010B5094BFF
:1007B0001B68002B0BD1084AD90004688C50406894
:1007C000521850600133034A1360002010BD01200D
:1007D000FCE7C046C40C2020C80C202010B5002027
:1007E000002400E00134094B1B68A3420DD9E3004B
:1007F000074A9B589B68002BF4D098470128F1D1F9
:10080000E400034B1C19034B1C6010BDC40C2020DA
:10081000C80C2020D00C202010B52D4B1B681B6865
:10082000DB68002B0FD098471038C3B2072B45D890
:100830009800284B1B589F46254B1B685B681B681C
:10084000002B00D0984710BD214B1B685B685B688C
:10085000002BF8D09847F6E71D4B1B685B689B6838
:10086000002BF0D09847EEE7194B1B685B68DB68FC
:10087000002BE8D09847E6E7154B1B685B681B69BF
:10088000002BE0D09847C046DDE7114B1B685B6842
:100890001B6A002BD7D09847D5E70D4B1B681B6808
:1008A0001B69002BCFD079209847CCE7084B1B68F9
:1008B0005B685B69002BC6D09847C4E7044B1B6894
:1008C0001B681B69002BBED01F209847BBE7C046A2
:1008D000D00C20202862000010B500F0DFFE10BD13
:1008E00010B582B06A460D4B03CB03C2792000F0ED
:1008F000CDFA082000F0CAFA212000F0C7FA00243F
:1009000004E06B46185D00F0C1FA0134072CF8D9F9
:10091000792000F0BBFA02B010BDC046486200006A
:10092000F8B500F009FA002803D01F2000F0AEFA55
:100930001CE0792000F0AAFA1B4A13781B025178B8
:100940000D001D4311701B0A5370EE0807272F403E
:10095000002E0CD1002F1AD1802280205200124983
:10096000000200F0EFF9792000F090FAF8BD0024C1
:10097000B442EFD0E00002300B4BC0181722082120
:1009800000F04CFA792000F081FA0134F0E7E81B1E
:100990000230054D40191722082100F03FFA792056
:1009A00000F074FAD8E7C046080D202010B5040006
:1009B000094A13781B06517809040B439178090200
:1009C0000B43D0781843206000F044F9002801D18F
:1009D0001F3010BD7920FCE7080D202000B583B042
:1009E00000F0AAF9002804D01F2000F04FFA03B04D
:1009F00000BD792000F04AFA01A8FFF7D7FF1F28B1
:100A00000AD000F071FB002809D0792000F03EFAEE
:100A1000019800F093F9EAE700F038FAE7E71F20C1
:100A200000F034FAE3E70000F0B583B000F084F999
:100A3000041E04D01F2000F029FA03B0F0BD01A865
:100A4000FFF7B4FF1F2815D0792000F01FFA184BCC
:100A50001D790135EF0807262E40072D0DD8002EF1
:100A60001AD12A001249019800F04AF9792000F0C1
:100A70000DFAE2E700F00AFADFE7BC42EFD0E0004F
:100A80000B4BC0181422082100F0C8F9792000F09F
:100A9000FDF90134E4B2F0E7A81B054E80191422D9
:100AA000082100F0BBF9792000F0F0F9D9E7C04641
:100AB000080D2020F0B5CE46474680B583B000F043
:100AC0003BF9071E07D01F2000F0E0F903B00CBC73
:100AD00090469946F0BD01A8FFF768FF1F280FD088
:100AE000792000F0D3F9284B1B790133DA089046BE
:100AF00007221A409146019800F0CEF8060021E046
:100B000000F0C4F9E2E70830310000F0E1F831000C
:100B1000019800F0DDF81D4B18550134E4B2019B3B
:100B200001330193013D002D04D00198184B9842E8
:100B3000EDD8E8E70821154800F024FA01235B42CC
:100B40009C46E0444346002B02D03C000825EAE7DF
:100B50004B46002B16D1792000F098F9B6E731000A
:100B6000019800F0B5F8094BD8550137FFB2019B49
:100B700001330193013C002CF1D14946034800F0B8
:100B800001FAE8E74C46F6E7080D2020080E202081
:100B9000EFFF010010B5792000F078F90548342303
:100BA000037003334370022100F0ECF9792000F068
:100BB0006DF910BD080E202010B5792000F066F9FF
:100BC000212000F063F905480023037043700221DF
:100BD00000F0D8F9792000F059F910BD080E202056
:100BE000004870475400202070B5184B1968002940
:100BF0002AD1174B4A00541824010568E5501B19E7
:100C000042685A6082689A60C268DA6002691A6152
:100C100042695A6182699A61416A5962C16AD962BC
:100C20009047082805D0094A136801331360002053
:100C300070BD064B1A6853009B181B01044AD31859
:100C4000802292025A60EEE70120F1E7D40C2020C6
:100C5000D80C2020002300E001330D4A12689A428C
:100C600013D95A00D21812010A4952588242F3D8B5
:100C70005A00D21812018A1852688242ECD35A00E4
:100C8000D3181B01CB18D86800E000207047C0467D
:100C9000D40C2020D80C20200100002000E00130DE
:100CA000094B1B6883420DD943001B181B01074ADF
:100CB0009B588B42F3D843001B181B01D3185B6869
:100CC0008B42ECD37047C046D40C2020D80C202097
:100CD00010B5094B1B688B4209D94B005918090103
:100CE000064B59180B69002B03D0984700E00020F1
:100CF00010BD0020FCE7C046D40C2020D80C2020DA
:100D000070B506000C001500FFF7C6FF084B1B6806
:100D100083420BD9430018180001064B1818436989
:100D2000002B03D02A0021003000984770BDC04638
:100D3000D40C2020D80C20200020704710B500F0E3
:100D400087F910BD70B50C001500FFF7A5FF0A4B21
:100D50001B6883420BD9430018180001074B181871
:100D6000C36A002B05D029002000984700E001202D
:100D700070BD0120FCE7C046D40C2020D80C2020F8
:100D800010B50021014800F015FA10BD0080504058
:100D900010B5024800F0A0FA10BDC04600805040D7
:100DA00010B5FFF7EDFF10BD30B583B0002501246D
:100DB000002C11D0144B1A00803A190084390A20F3
:100DC0000090124800F0D6FA0400FFF785FD0135C7
:100DD000642DEDDD0025EBE7FFF77EFD0C4B5B6836
:100DE000D8B20C4A5360002306E0094AD218117A9F
:100DF000094AD1540133DBB2054988228A5C9A4200
:100E0000F3D803B030BDC046781020200080504099
:100E1000F00F20209C002020080D2020F0B583B08A
:100E200007000E001500164B00225A60002403E054
:100E30000134642C00DD0024124B1A00803A1900A2
:100E400084390A200090104800F094FA0028EFD16D
:100E50000B4B5B68AB42EBD1FFF73EFD084B5B6889
:100E6000AB420AD003B0F0BD054AD218127AFA5448
:100E70000133DBB2B342F7D3F4E70023FAE7C0460D
:100E8000F00F2020781020200080504010B582B054
:100E9000124A01238821535451682031516048245B
:100EA00010534832009300230D4800F0F3FA002459
:100EB00004E00B4800F0E4FA01231840002804D0B5
:100EC0000134642CF5DD0024F3E7FFF705FD034A48
:100ED0005368203B536002B010BDC0469C002020E8
:100EE0000080504030B585B0002302930393204B1F
:100EF0001A00803A19008439642000901D4800F0DF
:100F000039FA00282CD11C4B5B68DAB21B494B60C4
:100F1000162A01D0002424E002AB17490A00083247
:100F2000180030CA30C000229A71C87B03001E3BF3
:100F3000DBB2092B1AD80A21FFF748F9C9B20529F3
:100F400001D000240DE00E4902A8FFF745F9002862
:100F500001D0002405E07930FFF798FF012400E07C
:100F60000024FFF7B9FC200005B030BD0024F8E7ED
:100F70007810202000805040F00F20209C0020207E
:100F80005062000070B582B00E00164B8822995452
:100F90005968203159600023B34207D2C55C1A005A
:100FA000243252000F4C15530133F5E7009600230D
:100FB0000D4A0E4800F06EFA002404E00B4800F0E1
:100FC0005FFA01231840002804D00134642CF5DDB9
:100FD0000024F3E7FFF780FC024A5368203B53608C
:100FE00002B070BD9C002020E40020200080504012
:100FF000054B1B78002B04D1034B01221A700020F3
:10100000704701204042FBE7080F2020007870471E
:10101000F8B506000F001500530702D007239D43C3
:101020000835002402E000F09BFC0834AC420BD2EF
:1010300000F098FC3A19A119044800F09AF840B25F
:101040000028F0D0C046EEE7F8BDC04600D00C4006
:1010500010B50400FFF79CFE00F086FC084B002250
:101060001A605A609A60236883F30888236883F3C0
:101070000988BFF36F8F034B9C606368984710BD6E
:1010800010E000E000ED00E0F0B5C64600B5050058
:101090000E000788023500F065FC00239846002406
:1010A0000BE089020F4800F04EF840B2002802D051
:1010B00001239C46E04401350134BC4207D2730849
:1010C000A34204D929781F29EBD8C046F3E700F0E2
:1010D00047FC4346002B03D0012004BC9046F0BDE2
:1010E0000020FAE700D00C4010B580200002FFF786
:1010F000B1FD012818D180231B0219684B1C15D0A3
:101100000A000023FE2000060321494212184B4129
:1011100007490C68002101208B4202DC02D1A24267
:1011200000D9002040B200E0002010BD0020FCE704
:101130005801202010B500F071FD10BD10B500F071
:1011400063FE40B210BD70B504000D008022920015
:10115000FFF7F0FF40222900200000F0E9FC0328FF
:1011600005D0042801D0012070BD0238FCE7002022
:10117000FAE770B504000D00160080229200FFF718
:10118000D9FF32002900200000F030FD032803D0F1
:1011900004280CD0012070BD320029002000FFF788
:1011A000CDFF032801D00120F5E70020F3E7023846
:1011B000F1E7000030B58BB004000D00354BEC2298
:1011C00086219950043234499950344B984245D184
:1011D000012D49D8324B1B78002B4BD1F223DB0178
:1011E0000122C2502F4900F041FE6946200001F063
:1011F0004BFD200000F05AFE0028FAD0012120000B
:1012000000F078FE200000F08BFE0128FAD126497C
:10121000200000F099FE2549200000F085FF002DF8
:101220002ED0012D31D02249200001F0CDF8214AE5
:101230000021200001F0B8FB1F49200001F034FA22
:101240000021200000F056FE200000F069FE00287A
:10125000FAD1134B01221A700BB030BD174B184A4C
:10126000B921184802F09CF9174B154ABA211548C4
:1012700002F096F9154B124ABB21124802F090F980
:101280001349200000F0FAFFCDE71249200000F0DA
:10129000F5FFC8E70080424086000400008050400F
:1012A000090F202038630000CC012020A00120205D
:1012B000000220203C630000FFFFFF1F5862000077
:1012C000F0620000686200008C620000B4620000FE
:1012D000800120206001202010B504001A4B9842A4
:1012E00024D11A4B1B78002B27D0194B194AC25016
:1012F000102000F051FB0023F222D201A3508022E3
:10130000154940208850BFF34F8FBFF36F8FD02116
:10131000C9019820800560500C490B700F4BEC21DF
:101320005A5070320E499950002010BD83210D4B48
:101330000D4A49000D4802F033F908210C4B0A4AC6
:10134000FF310A4802F02CF900805040090F20209C
:1013500004680000030000B100E100E000804240AA
:101360008000040058620000006300006862000012
:10137000CC620000F0B5CE46474680B583B08946C2
:1013800090461F000A9E354B98421CD1344B1B7867
:10139000002B1FD0334B00225A6000F0B3FA050037
:1013A000304B5B68002B1CD100F0ACFA401BB04204
:1013B0004CD22A4C2B49200001F090FB2A492000F6
:1013C00001F036FBECE7D621284B294A4900294891
:1013D00002F0E6F8D721284B254A4900254802F0BB
:1013E000DFF8204C0023236023681C4D234A009221
:1013F00000220121280001F01FFA2168A2682800BC
:1014000001F0CEFB002827D11C4B1A7D3A709B6857
:10141000012B08D0194B1B689B0C5B055B0D4A46E2
:10142000136000230DE0154B4A461B681360F8E774
:101430001A00143252001149525A4146CA5401331B
:10144000DBB23A789A42F3D8002000E0032003B0E0
:101450000CBC90469946F0BD0020F8E70080504053
:10146000090F20202411202078112020586200002C
:101470002463000068620000CC6200000C0F202092
:1014800010B501F0EFFBC0B2012801D0012010BD62
:101490000020FCE7F0B5C64600B5060017009846E8
:1014A000069A374B98420FD1364B1B78002B12D03F
:1014B000082A17D880231B0199421AD3324B0120E6
:1014C00098601960002123E09321304B304A490095
:1014D000304802F065F828212F4B2D4AFF312D4866
:1014E00002F05EF894212D4B294A4900294802F068
:1014F00057F8254B0020986089041960E2E74B00FB
:10150000D85B0D0010356D001F4C6419A0800131AF
:101510009142F4D31C4B1A61C04642460021300070
:1015200001F0EEF84146300001F052F9431C25D09D
:1015300000F0E8F91A4B18601A4B02221A700BE0FF
:10154000C046184B187840B204BC9046F0BD30003D
:10155000FFF796FF134B1870124B1B78002BEFD040
:10156000104B1B78012BEBD000F0CCF90C4B1B6817
:10157000C01A0228EBD9C0460320E5E70120E3E7C3
:1015800000805040090F2020600220205862000097
:101590001463000068620000CC620000E462000096
:1015A000D83120200403202040284DD883002A4A27
:1015B000D3589F463020002301E030200223274AE1
:1015C0001278002A43D10343C92000061843244B54
:1015D000882252019850234ABE2109069950802240
:1015E00012019B58DB0735D51F4A204BD3581B05EA
:1015F000FAD51A4B01221A70002027E0302003236D
:10160000DDE730200423DAE730200523D7E7302058
:101610000623D4E730200723D1E720200123CEE79B
:1016200020200223CBE70323C9E720200423C6E7B9
:1016300020200523C3E720200623C0E7202007231E
:10164000BDE730200123BAE7012040427047012066
:101650004042FBE70320F9E74C630000B40F202071
:10166000002008400411000000F00A4004120000AD
:10167000084B1B78002B0AD0074A80231B019821B6
:101680008905D150034B00221A70002070470120B9
:101690004042FBE7B40F202000200840054A064BDB
:1016A000D358012B01D001207047044BA721D15002
:1016B0000020F9E7002008400C110000081100008C
:1016C000074A084BD15808480140D150D15803303F
:1016D000FF308143D150054B00221A707047C0463D
:1016E00000F00A4008110000FFFEFFFFB50F2020A8
:1016F000114B1B78012B1AD0104B984219D101388D
:1017000080235B0498420DD20D4A50600D48036A55
:101710001B021B0AC02109060B43036200239360CE
:1017200007331360044B01221A70002003E00120EC
:1017300001E0012040427047B50F202080BB00002F
:1017400010E000E000ED00E010B50949094A0A4B3D
:10175000CA500A4B0A481A500A4AD020C0010A50FF
:10176000802109015A50102000F016F910BDC04622
:1017700000805040030000B10468000000200840D1
:10178000040800000100002610B5032902D0062934
:1017900000D08FE0022802D0042800D08DE0032979
:1017A00007D0062922D0022825D0042855D00020B1
:1017B00010BD434B8A2252010239995041490A69AE
:1017C000042422430A6140495A58404C22405A504E
:1017D0003F4A002199503F4A116880239B004B40AB
:1017E000F024240123404B401360DCE7344A384B9B
:1017F0000021D150D7E7324A354B0021D150354C2A
:10180000216880239B004B40F020000103404B40A7
:10181000236031490B68032083430B602F4BD15861
:1018200002388143D150D1582D480140D1508230E7
:10183000FF3001220A21800101F078FE294801F0E1
:10184000ABFD216810224A40302313404B402360F7
:10185000002001F03BFE0020AAE71F4A1368032185
:101860008B431360164C1D4BE25802398A43E250F9
:10187000E2581B490A40E2501A4801F08DFD1A4A0D
:101880001168A023DB014B40F020000203404B40D5
:1018900013600D49605880235B0103436350134973
:1018A0006358102003436350136811490B401360C1
:1018B00000207DE7012040427AE70120404277E79F
:1018C00000F00A4000ED00E004110000FFFFDFFF20
:1018D0000813000004010B4000010B400811000038
:1018E000FFFEFFFF5064000038010B403C11000078
:1018F000FFFDFFFF024A1368013313607047C046C3
:10190000E4312020014B18687047C046E4312020A4
:1019100010B584B00400FFF7F5FF03900023029395
:10192000FFF7F0FF0190029BA34207D2019B039AAD
:101930009B1A0293FFF7E6FF0190F4E704B010BD95
:1019400010B5FFF701FF03210220FFF71DFF034839
:10195000FFF7CEFE0820FFF727FE10BD80BB00007A
:1019600062B6704772B6704710B5FFF781FEFFF799
:10197000A7FEFFF7F7FF10BD044B9822520100218C
:101980009950034A034999507047C04600F00A40F5
:1019900004130000010000E480B584B000AF78605B
:1019A0007A68931E043BC046FCD2FB60C046BD462D
:1019B00004B080BD80B584B000AFF860B9607A60D3
:1019C000FA68BB681A4305497B681A4398235B0190
:1019D000CA50C046BD4604B080BDC046000040406D
:1019E00080B500AF044A98235B01D3580722134007
:1019F0001800BD4680BDC0460000404080B582B0A2
:101A000000AFFFF7EDFF03007B60042200210120FF
:101A1000FFF7D0FF084B9B699AB2BB1C1205120D51
:101A20001A80064998235B017A68CA50BB1C1B8840
:101A30001800BD4602B080BD0000C4410000404017
:101A400080B582B000AFFFF7CBFF03007B600422BC
:101A500000210120FFF7AEFF0A4B9B691B0BDBB295
:101A600003221340DAB2FB1C01321A700649982394
:101A70005B017A68CA50FB1C1B781800BD4602B097
:101A800080BDC0460000C4410000404080B500AFAA
:101A900000231800BD4680BD80B582B000AF7860DD
:101AA00039607A6889235B013968D150C046BD46E8
:101AB00002B080BD80B582B000AF786039603B680D
:101AC0009B0A1800BD4602B080BDB0B588B000AF1B
:101AD000786039601B257C19FFF7B2FF0300237083
:101AE000FFF78CFF03007B613A687B6811001800E8
:101AF000FFF7E0FF03003B617B191B78012B0FD937
:101B00007B191B7819007869FEF7DAFA0300FB608D
:101B10003B69F9681800FEF759FB0B00FB6101E017
:101B20003B69FB61FB691800BD4608B0B0BD000011
:101B300080B584B000AFF860B960FB1D1A70FB1D62
:101B40001B7802221343DBB21900FB68084A995044
:101B5000BA68FB6811001800FFF79EFFFB681800C9
:101B600004F00AFB03001800BD4604B080BDC04667
:101B70000411000080B584B000AFF860B9607A60ED
:101B8000FB68084A01219950FB6807497A685A5056
:101B9000BA68FB6811001800FFF77EFFC046BD461B
:101BA00004B080BD041100002411000080B584B091
:101BB00000AFF860B9607A603B607A68B968FB682A
:101BC0001800FFF7D7FF3B681A68FB6805495A50B1
:101BD0003B685A68FB6804495A50C046BD4604B089
:101BE00080BDC046301100003411000080B584B0C3
:101BF00000AFF860B9607A607B68074AB968F86836
:101C0000FFF7D4FFFB68180004F0B6FA03001800D1
:101C1000BD4604B080BDC046FF010000B0B58AB02B
:101C200000AFF860B960BB1D1A80BA68FB6811008C
:101C30001800FFF73FFF03003B62BA68FB68110022
:101C40001800FFF742FF0300FB611B257C19FFF71B
:101C5000F7FE03002370FFF7D1FE03007B61002332
:101C60007B62BB1D1A8880239B009A4200D06CE0E7
:101C7000FFF70CFF031E14D07B191B78012B10D922
:101C80007B695B083A6A9A4205D97B695B083A6AC4
:101C9000D31A7B6207E07B695B083A6AD3187B62E0
:101CA00001E03B6A7B627B6A1F2B0ED801227B6AB4
:101CB0009A4013003B61FB68314A9B583A69D24312
:101CC0001A40FB682E495A5055E0FB69FF2B25D876
:101CD000FFF7B6FE0300012B10D1FB69203BDB08A8
:101CE00001229A4013003B61FB68264A9B583A69DF
:101CF000D2431A40FB6823495A503CE0FB69DB0899
:101D000001229A4013003B61FB681E4A9B583A69C6
:101D1000D2431A40FB681B495A502CE0FA69FF2352
:101D20005B009A4227D8FB69013BFF3BDB0801229D
:101D30009A4013003B61FB68134A9B583A69D243AF
:101D40001A40FB6810495A5015E0BB1D1A888023C1
:101D5000DB009A420FD13B6A1F22134001229A40B6
:101D600013003B61FB68094A9B583A69D2431A4009
:101D7000FB6806495A50C046BD460AB0B0BDC046D1
:101D8000D0110000D4110000D81100001012000082
:101D900080B584B000AFF860B9607A60FB68084A2B
:101DA00003219950FB6807497A685A50BA68FB6862
:101DB00011001800FFF770FEC046BD4604B080BD9C
:101DC000041100002411000080B584B000AFF86059
:101DD000B9607A603B607A68B968FB681800FFF701
:101DE000D7FF3B681A68FB6805495A503B685A6838
:101DF000FB6804495A50C046BD4604B080BDC04689
:101E0000301100003411000080B584B000AFF860DC
:101E1000B9607A607B68074AB968F868FFF7D4FF51
:101E2000FB68180004F0A8F903001800BD4604B0D0
:101E300080BDC046FF01000080B586B000AFF860ED
:101E4000B9607A60FB681B687B617B68DA437B69F9
:101E500013407B61BB687A681A407B691A43FB6850
:101E60001A60C046BD4606B080BD000080B582B095
:101E700000AF786039600A4B0A4A98183B681B88A3
:101E8000190080235B001A00FFF7D6FF3B689B78A0
:101E900019007B68044A9950C046BD4602B080BD17
:101EA00000F00A40381100000479000080B584B0C9
:101EB00000AF78607B680E4A944663440122022199
:101EC000180001F07CF90300BB60BB68012B04D152
:101ED0000F23FB1801221A7003E00F23FB180022C6
:101EE0001A700F23FB181B781800BD4604B080BD84
:101EF0000872000080B582B000AF786039607B68FE
:101F0000064A9446634418003B680022012101F010
:101F100037F9C046BD4602B080BDC046187000000B
:101F200080B582B000AF78607B68064A944663440F
:101F300000220121180001F042F903001800BD46FB
:101F400002B080BD1870000080B584B000AF78602A
:101F500039607B686A4A94466344180001F0F8F8D7
:101F60000300BB60BB68102293431A003B689B6967
:101F70001B0110210B401343BB60BB68202293431D
:101F80001A003B68DB695B0120210B401343BB60F7
:101F9000BB68082293431A003B681B6ADB000821D8
:101FA0000B401343BB607B68554A944663441A0058
:101FB000BB681900100001F0D7F87B68180000F02A
:101FC000B7FE7B684F4A94466344180001F0C0F89E
:101FD0000300BB60BB684C4A1A403B681B6819028F
:101FE00080235B000B401343BB60BB68474A1A4029
:101FF0003B685B68590280239B000B401343BB6026
:10200000BB68434A1A403B689B6899038023DB0105
:102010000B401343BB60BB683E4A1A403B68DB6819
:10202000590380239B010B401343BB60BB683A4AB2
:102030001A403B681B69190380235B010B40134363
:10204000BB60BB68402293431A003B685B699B01FD
:1020500040210B401343BB607B682A4A944663448B
:102060001A00BB681900100001F07EF83B689B6AFB
:102070007F2B38D83B68DB6A7F2B34D83B685B6AA0
:10208000FF2B30D87B68254A9446634418003B6890
:102090009B6A00227F2101F073F87B681F4A9446F7
:1020A000634418003B68DB6AFE22D101082201F07C
:1020B00067F87B681A4A9446634418003B685B6A79
:1020C0000022FF2101F05CF87B68164A94466344C5
:1020D00018003B681B6B80221104172201F050F896
:1020E0000023FB6002E001235B42FB607B68180079
:1020F00000F032FEFB681800BD4604B080BDC0464B
:102100000472000018700000FFFEFFFFFFFDFFFFDC
:10211000FFBFFFFFFFDFFFFFFFEFFFFF4870000083
:10212000147000000C70000080B584B000AF7860BF
:1021300039607B68180000F0FBFD7B684B4A9446D1
:10214000634418003B681B680522202101F018F841
:102150007B68464A9446634418003B685B680222E9
:10216000042101F00DF87B68E122D201944663441A
:1021700018003B68DB690022012101F001F87B684F
:10218000E122D2019446634418003B681B6A012295
:10219000022100F0F5FF7B68E122D20194466344FE
:1021A00018003B685B6A02220C2100F0E9FF7B68A3
:1021B000E122D2019446634418003B689B6A0422E2
:1021C000302100F0DDFF3B689B680F2B41D83B6856
:1021D0005A6980235B029A423BD27B68244A944628
:1021E000634418003B68DB680022032100F0C8FF4D
:1021F0007B681F4A9446634418003B689B68013B18
:10220000F0221103102200F0BBFF7B68194A9446AC
:10221000634418003B681B690122062100F0B0FFEF
:102220007B68144A9446634418003B685B69124912
:10223000102200F0A5FF7B680E4A94466344180004
:102240003B689B690022012100F09AFF0023FB609C
:1022500002E001235B42FB607B68180000F07CFD1C
:10226000FB681800BD4604B080BDC0461870000071
:1022700020700000287000000000FFFF80B584B0CF
:1022800000AF786039607B68180000F051FD3B6852
:10229000DB687F2B3ED83B689B687F2B3AD83B6836
:1022A0005B68FF2B36D83B681A6880239B009A42F4
:1022B00030D27B68414A9446634418003B68DB682F
:1022C000FE221106192200F05BFF7B683B4A944610
:1022D000634418003B689B6800227F2100F050FF98
:1022E0007B68364A9446634418003B685B68FF226B
:1022F0001102082200F044FF7B68304A9446634490
:1023000018003B681B682E49102200F039FF00239B
:10231000FB6002E001235B42FB60FB68002B43D1C2
:102320003B68DB690F2B3CD83B689B690F2B38D887
:102330003B685B691F2B34D83B681B691F2B30D867
:102340007B68204A9446634418003B68DB6900229E
:102350000F2100F015FF7B681A4A94466344180069
:102360003B689B690422F02100F00AFF7B68154A54
:102370009446634418003B685B69F82251010822C7
:1023800000F0FEFE7B680F4A9446634418003B68E9
:102390001B69F8225103102200F0F2FE0023FB60BB
:1023A00002E001235B42FB607B68180000F0D4FC74
:1023B000FB681800BD4604B080BDC0461C7000001C
:1023C0000000FF010C70000080B584B000AF7860A1
:1023D00039600023BB607B68180000F0A9FC3B68F3
:1023E0005B68002B17D07B68A54A944663441800AD
:1023F0003B681B689B08A349022200F0C1FE7B6872
:102400009F4A9446634418003B685B68FF221104AE
:10241000102200F0B5FE3B68DB68002B17D07B680C
:10242000994A9446634418003B689B689B08954909
:10243000022200F0A5FE7B68934A9446634418008C
:102440003B68DB68FE22D103102200F099FE3B6856
:102450005B6B002B3AD07B688C4A9446634418002F
:102460003B681B6B9B088749022200F089FE7B6852
:10247000864A9446634418003B685B6BFE22D10396
:10248000102200F07DFE7B68804A94466344180069
:102490003B689B6BFE22D105182200F071FE7B6821
:1024A0007A4A9446634418003B68DB6B802211062D
:1024B0001F2200F065FE7B68754A9446634418004D
:1024C0003B689B6D0022072100F05AFE3B685B6C65
:1024D000002B3AD07B686F4A9446634418003B68EF
:1024E0001B6C9B086749022200F04AFE7B68694A20
:1024F0009446634418003B685B6CFE22D1031022B3
:1025000000F03EFE7B68634A9446634418003B68D3
:102510009B6CFE22D105182200F032FE7B685D4ADA
:102520009446634418003B68DB6C802211061F222E
:1025300000F026FE7B68564A9446634418003B68C8
:10254000DB6D0422702100F01BFE7B68524A94462A
:10255000634418003B681B6D9B084A49022200F047
:102560000FFE7B684A4A9446634418003B685B6DE3
:10257000E022D100082200F003FE3B689B6A002B9A
:1025800023D07B68454A9446634418003B685B6AE5
:102590009B083C49022200F0F3FD7B683F4A9446C9
:1025A000634418003B689B6AFC229103102200F0F0
:1025B000E7FD7B68394A9446634418003B68DB6A50
:1025C000FC229105182200F0DBFD3B685A693B684C
:1025D0009B69D318BB60BB68202B45D83B685B69FF
:1025E000002B03D13B689B69002B3DD07B682C4AB4
:1025F0009446634418003B681B699B0821490222EA
:1026000000F0BEFD7B68264A9446634418003B6890
:102610005B69FC229103102200F0B2FD7B68204A26
:102620009446634418003B689B69FC22910518227C
:1026300000F0A6FD7B681A4A9446634418003B6884
:10264000DB698022D1051E2200F09AFD7B68154AC5
:102650009446634418003B681B6A0022072100F07F
:102660008FFD0023FB6002E001235B42FB607B687F
:10267000180000F071FBFB681800BD4604B080BD77
:1026800084700000FCFF000088700000A070000053
:10269000BC700000B0700000AC700000F070000072
:1026A000C0700000C870000080B584B000AF7860D2
:1026B00039603A6880239B059A4214D27B681800DF
:1026C00000F036FB7B680C4A9446634418003B6874
:1026D0000A49002200F054FD7B68180000F03CFB22
:1026E0000023FB6002E001235B42FB60FB681800F3
:1026F000BD4604B080BDC04690700000FFFFFF1FC4
:1027000080B58AB000AFF860B9607A603B600023A2
:10271000FB610023BB6100237B6100237B620023FC
:102720003B62BB68002B03D17B687B6201233B6269
:10273000BB68012B0ED1FB68214A94466344180004
:10274000F8235B031022190000F039FD03007B62BF
:1027500001233B623B6A012B2ED1FB68194A944648
:1027600063441800184B0222190000F028FD0300F2
:10277000FB61FB68154A9446634400220721180058
:1027800000F01DFD0300BB61FB699B00FB61BB69A1
:10279000180000F0C5FC0300BB61BB699B00BB6176
:1027A000BB697A6A5343FA69D3187B61FB683A685C
:1027B0007969180000F0C0FBC046BD460AB080BD74
:1027C000C4700000C0700000FCFF0000C870000072
:1027D00080B584B000AF786039603B681F2B20D88B
:1027E0007B68144A94466344180000F0B1FC03006F
:1027F000BB6001223B689A401300BA681343BB6078
:102800007B68180000F0A8FA7B680A4A9446634483
:102810001A00BB681900100000F0A6FC0023FB6042
:1028200002E001235B42FB60FB681800BD4604B078
:1028300080BDC046D070000080B58AB000AFF8609F
:10284000B9607A603B6000237B6200233B62002317
:102850007B610023FB610023BB61BB68002B1CD1A3
:10286000FB684A4A944663441800494B0222190007
:1028700000F0A5FC03007B62FB68464A9446634473
:102880001800E023DB000822190000F098FC030088
:102890003B627B68BB610123FB61BB68012B54D1A8
:1028A0003B68002B03D03B68012B27D04EE0FB6830
:1028B000394A944663441800354B0222190000F04F
:1028C0007EFC03007B62FB68324A9446634400222C
:1028D0000721180000F073FC03003B62FB682F4ADD
:1028E000944663441800FC239B010822190000F061
:1028F00066FC0300BB610123FB6127E0FB68284AFB
:10290000944663441800224B0222190000F057FC41
:1029100003007B62FB681F4A9446634404227021D3
:10292000180000F04CFC03003B62FB681D4A944613
:1029300063441800FC239B010822190000F03FFCAF
:102940000300BB610123FB6100E0C046FB69012B72
:1029500017D17B6A9B007B623B6A180000F0E0FBAA
:1029600003003B623B6A9B003B623B6ABA6953438C
:102970007A6AD3187B61FB683A6B7969180000F0BA
:10298000FFF9C046BD460AB080BDC046AC7000002D
:10299000FCFF0000BC700000A0700000A4700000EC
:1029A000B0700000B470000080B588B000AFF8606F
:1029B000B9607A60FB681C4A9446634418001B4B5C
:1029C0000222190000F0FBFB0300FB61FB699B0086
:1029D000FB61BB689B00FA69D318BB6100237B6174
:1029E0007B681B687A6913437B617B685B681B04A7
:1029F0007A6913437B617B689B68DB067A691343C2
:102A00007B617B68DB689B077A6913437B61FA68AB
:102A1000BB69D3187A691100180000F0A5FBC04605
:102A2000BD4608B080BDC04684700000FCFF0000B9
:102A300080B584B000AF786039607B68264A9446E0
:102A40006344180000F084FB0300FB60FB6807226E
:102A50001A403B681A60FB68DB0803221A403B6897
:102A60005A60FB685B0901221A403B689A60FB6868
:102A70009B0901221A403B68DA60FB68DB090122EE
:102A80001A403B681A61FB681B0A07221A403B6820
:102A90005A61FB68DB0A01221A403B689A61FB68B5
:102AA0001B0B01221A403B68DA61FB685B0B0122B9
:102AB0001A403B681A62FB689B0B01221A403B6874
:102AC0005A62FB681B0C7F221A403B689A62C04620
:102AD000BD4604B080BDC0464470000080B584B0DF
:102AE00000AF786039603B681B68002B02D0012B77
:102AF00027D04DE07B68284A94466344180000F0D4
:102B000027FB0300FB60FB687F221A403B685A608A
:102B1000FB681B0A3F221A403B689A60FB681B0C4B
:102B20003F221A403B68DA60FB681B0E01221A4004
:102B30003B681A61FB685B0E01221A403B685A61D0
:102B400026E07B68154A94466344180000F000FBB9
:102B50000300FB60FB687F221A403B685A60FB68F9
:102B60001B0A3F221A403B689A60FB681B0C3F22FD
:102B70001A403B68DA60FB681B0E01221A403B6872
:102B80001A61FB685B0E01221A403B685A61C0461D
:102B9000C046BD4604B080BDA4700000B470000003
:102BA00080B586B000AFF860B9607A60BB68002B72
:102BB00003D0BB68012B22D043E0FB68254A944632
:102BC00063441800FE23DB031022190000F0F7FA1B
:102BD00003003B613A697B689A420CD3FB681E4A4A
:102BE0009446634418007B6800223F2100F0C8FA35
:102BF00000237B6129E001235B427B6125E0FB68C8
:102C0000164A944663441800FE23DB031022190081
:102C100000F0D5FA03003B613A697B689A420CD315
:102C2000FB680F4A9446634418007B6800223F21EA
:102C300000F0A6FA00237B6107E001235B427B6181
:102C400003E001235B427B61C0467B691800BD46FF
:102C500006B080BDA0700000A8700000B070000039
:102C6000B870000080B582B000AF78607B68054A1C
:102C700094466344180000F06BFA03001800BD4648
:102C800002B080BDD870000080B584B000AF78601D
:102C900039607B68E422D20194466344180000F056
:102CA00057FA0300FB60FB683F221A403B68DA607A
:102CB000FB681B0A07221A403B689A60FB681B0CE2
:102CC0001B051A0D3B685A60FB689A0F3B681A6037
:102CD0007B68E022D20194466344180000F038FA81
:102CE0000300FB60FB68FF221A403B681A61FB6827
:102CF0001B0AFF221A403B685A61FB681B0C0F221B
:102D00001A403B689A61FB681B0D0F221A403B6812
:102D1000DA61FB681B0E0F221A403B681A62FB68DF
:102D20001A0F3B685A62C046BD4604B080BD000021
:102D300080B582B000AF78607B68064A94466344F1
:102D4000180001230122022100F01AFAC046BD46F4
:102D500002B080BD1870000080B582B000AF78600E
:102D60007B68064A9446634418000023012202212E
:102D700000F006FAC046BD4602B080BD18700000E3
:102D800080B586B000AFF860B9607A6000233B611F
:102D900000237B61FA68BB68D318180000F0D8F9EB
:102DA00003003B613B69DB00DA087B681A603B6922
:102DB0005B0F01221A407B685A603B699B0F01221E
:102DC0001A407B689A603B69DA0F7B68DA60BB68FF
:102DD0000433BB60FA68BB68D318180000F0B8F978
:102DE00003003B613B691B041A0C7B681A613B6959
:102DF0001B0C0F221A407B685A613B691B0D012294
:102E00001A407B689A613B695B0D01221A407B681E
:102E1000DA613B691B0E7F221A407B681A623B69AC
:102E2000DA0F7B685A62BB680433BB6000237B61A6
:102E300038E0FA68BB68D318180000F089F903007D
:102E40003B613B699BB2FF22134099B27B687A6970
:102E500014325200D1523B691B0A9BB27A6901328B
:102E6000FF210B4099B27B6814325200D1523B696A
:102E70001B0C9BB27A690232FF210B4099B27B682E
:102E800014325200D1523B69190E7B69DA1C89B2A7
:102E90007B6814325200D152BB680433BB607B693B
:102EA00004337B617B685B69180000F021F9020044
:102EB0007B69D31A032B08D97B685B69180000F083
:102EC00017F902007B699342B3D17B685B691800F4
:102ED00000F00EF902007B69934229D0FA68BB68C2
:102EE000D318180000F034F903003B613B699BB232
:102EF000FF22134099B27B687A6914325200D15292
:102F00003B691B0A9BB27A690132FF210B4099B2DF
:102F10007B6814325200D1523B691B0C9BB27A6918
:102F20000232FF210B4099B27B6814325200D15219
:102F3000C046BD4606B080BD80B586B000AFF86023
:102F4000B9607A6000233B6100237B6100233B6111
:102F50007B681A687B685B685B071A437B689B68C1
:102F60009B071A437B68DB68DB0713433A6913430B
:102F70003B61FA68BB68D3183A691100180000F089
:102F8000F3F8BB680433BB6000233B617B681B69BB
:102F90001A047B685B691B051A437B689B695B05A8
:102FA0001A437B68DB69DB051A437B681B6A1B06D7
:102FB00013433A6913433B61FA68BB68D3183A6913
:102FC0001100180000F0D0F8BB680433BB60002388
:102FD0007B6139E000233B617A687B6910335B00D9
:102FE000D31804331B8819007B6901337A681033C6
:102FF0005B00D31804331B881B020A001A437B6949
:103000000233796810335B00CB1804331B881B0430
:103010001A437B690333796810335B00CB180433A0
:103020001B881B0613433A6913433B61FA68BB686C
:10303000D3183A691100180000F096F8BB68043301
:10304000BB607B6904337B617B681B69180000F0FF
:103050004FF802007B69D31A032B08D97B681B69E0
:10306000180000F045F802007B699342B2D17B68FA
:103070001B69180000F03CF802007B69934233D0D2
:1030800000233B617A687B6910335B00D3180433FB
:103090001B8819007B6901337A6810335B00D318F1
:1030A00004331B881B020A001A437B6902337968C8
:1030B00010335B00CB1804331B881B041A437B6955
:1030C0000333796810335B00CB1804331B881B066D
:1030D00013433A6913433B61FA68BB68D3183A69F2
:1030E0001100180000F040F8C046BD4606B080BD93
:1030F00090B593B000AF786008243A19074B1000E0
:10310000190040231A0000F09FFA3B197A689200D8
:10311000D3581800BD4613B090BDC046C86100002A
:10312000B0B58AB000AF786008217B18074A31CA71
:1031300031C331CA31C311CA11C37B187A689200F6
:10314000D3581800BD460AB0B0BDC04608620000A2
:1031500080B584B000AF78607B681B68FB60FB685B
:103160001800BD4604B080BD80B582B000AF786065
:1031700039607B683A681A60C046BD4602B080BDBF
:1031800080B586B000AFF860B9607A603B60FB68DC
:103190001B687B61BB68DA437B6913407B613A68DB
:1031A0007B689A401300BA6813407A6913437B61C5
:1031B000FB687A691A60C046BD4606B080BD80B51E
:1031C00086B000AFF860B9607A60FB681B687B610D
:1031D0007B69BA681A407B68DA4013007B617B69BF
:1031E0001800BD4606B080BD80B584B000AFF86061
:1031F000B9607A60FA68BB681A4305497B681A436C
:1032000098235B01CA50C046BD4604B080BDC0468D
:103210000000404080B500AF044A98235B01D358BA
:10322000072213401800BD4680BDC0460000404044
:1032300080B586B000AFF860B9607A60FB681B6843
:103240007B617B68DA437B6913407B61BB687A688A
:103250001A407B691A43FB681A60C046BD4606B037
:1032600080BD000080B500AF024A034BD358180060
:10327000BD4680BD00F00A400412000080B500AFDA
:10328000054A064BD3580449054A1340034A8B505C
:10329000C046BD4680BDC04600F00A40081100008F
:1032A000FFFEFFFF80B500AF054A064BD358044927
:1032B00001229343034A8B50C046BD4680BDC046A1
:1032C00000F00A400811000080B582B000AF020093
:1032D000FB1D1A700449FB1D1B78044A8B50C04625
:1032E000BD4602B080BDC04600F00A400C1100008F
:1032F00080B582B000AF7860064B074A94466344BD
:103300007968FF221800FFF793FFC046BD4602B060
:1033100080BDC04600F00A401011000080B582B0A8
:1033200000AF0200BB1D1A80064B074A9818BB1D50
:103330001B88C02292011900FFF77AFFC046BD46E4
:1033400002B080BD00F00A401011000080B500AF4F
:10335000054A064BD3580449802252051343034AB9
:103360008B50C046BD4680BD00F00A4010110000E1
:1033700080B500AF054A064BD3580449054A1340AF
:10338000034A8B50C046BD4680BDC04600F00A408F
:1033900010110000FFFFFFEFB0B584B000AF786000
:1033A000FFF76CFFC046FFF75DFF02008023DB01E3
:1033B0001A408023DB019A42F5D13D4B89246401F8
:1033C00018197B685B7E01221900FFF731FF384B2B
:1033D000384D58197B6820229B5C03221900FFF7A7
:1033E00027FFFFF717FF0300FB60042200210120E5
:1033F000FFF7FAFE7B685B6A2D491B682E4A8B50EB
:103400007B685B6A04332A491B682C4A8B502C4921
:1034100098235B01FA68CA50254B58197B68DB6911
:103420001A02FE23DB011340FE22D2011900FFF72E
:10343000FFFE1F4B18197B681B681A04F0231B033F
:103440001A407B685B681B031B041B0C1A437B68D8
:103450009B681902F0231B010B401A437B68DB6851
:103460001A437B681B691A437B685B6913437A685C
:10347000127E1343134A1900FFF7DAFE0C4A124B6F
:10348000D3580B498022520013430F4A8B50C04639
:10349000FFF7E8FE020080239B001A4080239B0078
:1034A0009A42F5D1C046C046BD4604B0B0BDC04644
:1034B00000F00A4024110000281100002C11000027
:1034C0000000404072FF0F000811000080B582B07C
:1034D00000AF0200FB1D1A70FB1D1B781800FFF7E0
:1034E000F3FEC046FFF7BEFE020080239B031A4096
:1034F00080239B039A42F5D10A4A0B4BD3580949C2
:10350000802252021343084A8B50C046FFF7AAFE9E
:10351000030010221340102BF8D1C046C046BD4610
:1035200002B080BD00F00A400411000080B582B0F6
:1035300000AF39601100BB1D021C1A807B1D0A1CE4
:103540001A70FFF7AFFEBB1D1B881800FFF7E6FEE1
:103550003B681800FFF7CCFE0F4A104BD3580E49BA
:10356000012213430D4A8B507B1D1B78002B0DD07D
:10357000FFF7ECFEC046FFF775FE020080235B00FC
:103580001A4080235B009A42F5D101E0FFF7F0FE7C
:10359000C046BD4602B080BD00F00A4008110000E0
:1035A00030B514001A000A4B05001B6885B0D868B6
:1035B000002C09D0074B019300912B00064902947F
:1035C00000F00EF801F062F8044B1C00F3E7C0466F
:1035D00008032020786400008864000084640000F0
:1035E0000EB400B582B003AB0100054804CB0068FF
:1035F000019300F0BFF802B008BC03B01847C04602
:103600000803202070B50C4D0C4E761BB61005D06B
:10361000002408CD01349847A642FAD1FDF752F8AC
:10362000074D084E761BB61005D0002408CD013496
:103630009847A642FAD170BD8867000088670000ED
:103640008867000088670000F0B5C64600B50F2AFD
:1036500041D903270D003E0005430C0003002E4016
:103660002F423DD11500103D2D09AC462D01A84635
:103670008044256867681D605F60A568E7689D6095
:10368000DF6010341F0010334745F2D165460F2329
:103690000C2401352D01491913404519144222D03B
:1036A0008C59AC5104369C1B032CF9D80324043BE1
:1036B0009B0801339B002240ED18C918561E002AB2
:1036C00006D00023CC5C1A00EC5401339642F9D1A9
:1036D00004BC9046F0BD0500561E002AF1D1F7E764
:1036E0000500561EEDE71A00F6E7C046F8B54E464F
:1036F0004546DE4657464B6EE0B5914606000D0046
:103700009B0433D513689A469368002B2CD05246FD
:1037100012689046524652689346970819D0002482
:1037200002E00134A74212D04246A300D158300033
:103730002A0001F045F9431CF3D14A460023936067
:1037400053603CBC90469946A246AB46F8BD4B46FA
:103750009B685A4603218A439B1A4A469360082273
:103760009446E244002BD2D10020E6E701F086FA2D
:10377000E3E7C046F0B5DE4657464E464546E0B55F
:10378000BFB08A4693461C0001900893002804D0DD
:10379000836B0293002B00D127E253465B6EDB075D
:1037A00000D537E153460C21595E53469A8993055B
:1037B00000D42BE180239B011A4209D10B435246CE
:1037C00051469381496E964A0A4051464A669AB2DA
:1037D00013073DD553461B69002B39D01A231340DC
:1037E0000A2B43D015AB129300235D46D3461493A6
:1037F000139315AE0C930B930E930D9305932B78A7
:10380000002B00D1A4E12C0004E063780134002BEC
:1038100000D1D9E0252BF8D1671BAC4200D0D7E00E
:103820002378002B00D193E1002310AAD370013B31
:103830000293002300276278651C0493013513006E
:10384000203B5A2B00D9F1E076499B00CB589F468C
:103850005146019800F0B0FE5346002801D000F018
:1038600044FE9A891A2313400A2BBBD153460E21DA
:103870005B5E002BB6DB53465B6EDB0703D4930520
:1038800001D400F008FE23005A465146019800F08A
:103890004DFE059074E1019B1800984601F092FBE3
:1038A000436818000D9302F03FFA0E900400404662
:1038B00001F088FB83680B93002C01D000F0F7FC2B
:1038C0002A78BBE720232A781F43B7E710231F433A
:1038D000089ABB0600D47BE1072307329A430133E1
:1038E0009C46944463460893536812680793069273
:1038F000002B01DA00F089FC029BB946013309D0A4
:1039000080239F43069A079B1100B946194301D1B2
:1039100000F04FFC069B079C002C00D046E3092BCF
:1039200000D943E36322069B25A930338B5401233E
:10393000039310ABB7249C464F466444029B039A02
:103940009946934200DA914610ABDB785A1E9341B8
:10395000994478E010231F43BB0600D42AE10723D3
:10396000089A07329A4318CA0693079408922E4B76
:103970001F40B9460023002210A9CA700298421CB9
:1039800000D1E3E180224F4697430699079A0C0045
:10399000144300D0D9E1002801D000F00DFD002B28
:1039A00001D000F00BFC4A4601331A4003924A460C
:1039B0003EAC1342C2D03021623325AAD15410ABA1
:1039C000B7249C466444B9E7671BAC4200D1BFE012
:1039D000149B3560FA18139B77600293013314929D
:1039E00013930836072B0BDD002A00D1DEE359467E
:1039F000019812AAFFF77AFE002800D090E215AED7
:103A0000059B9C46BC446346059309E75346986D65
:103A100001F0E0FA53460C21595E53469A89C9E6F3
:103A2000FFDFFFFFE8640000FFFBFFFF002A00D17B
:103A30008EE0002325AC227010AAD3700133994682
:103A400003930023029302231A003A400A923B4256
:103A500001D09C46E14484231A003A4009923B423B
:103A600006D14A46049B9B1A9846002B00DDDBE2F8
:103A7000139B14989C46591C10ABDB78002B0DD07F
:103A800010AB033333600123013073601490139142
:103A9000072900DD51E28C46083601310A9B002BD4
:103AA00019D011AB3360022302307360149013916C
:103AB000072900DC58E2002800D1A1E3594601980B
:103AC00012AAFFF713FE002800D029E2139B1498D6
:103AD0009C46591C15AE099B802B00D171E1029BBD
:103AE000039A9B1A9A46002B00DDC9E1039B3460C0
:103AF0009C466044736014901391072900DC5EE1DA
:103B0000002800D1E4E25946019812AAFFF7EEFD21
:103B1000002800D004E2149815AE7B0705D54A466C
:103B2000049B9C1A002C00DDDBE2049B4B4500DA71
:103B30004B46059A94469C4463460593002800D062
:103B4000E6E1002313932B7815AE002B00D05AE644
:103B5000149BDA460293002B01D000F0B7FC00233F
:103B6000139353465B6EDB0700D5DFE153469B8919
:103B70009A0501D400F018FC5B0601D500F0C0FCEA
:103B800005983FB03CBC90469946A246AB46F0BD76
:103B9000303A280000241100A3001B195B00CC1848
:103BA00003001A7801301100303905000929F3D9D2
:103BB000049444E6FB0600D551E37B0600D44BE3B6
:103BC000089A08CA9BB20693002308920793CEE690
:103BD000FB0600D54EE37B0600D448E308CA1BB2BF
:103BE0000693DB170793089282E600F05DFED4E5AA
:103BF000089B10AA10CB98460023D370002C01D14B
:103C000000F0F4FB029A531C00D18AE3002120004B
:103C100001F032FD002801D100F043FC031B0393A7
:103C2000434608930023029388E6089A25AC08CA05
:103C300010A923700023CB70013399460892039397
:103C4000FFE6089B04CB0492002A00DBFDE2049A05
:103C500008935242049204232A781F43EEE510236E
:103C60001F43B9464B469B0600D4ADE20723089A92
:103C700007329A4318CA06930794089201237AE6FA
:103C80002A78682A00D1A3E340231F43D6E52B23DB
:103C900010AAD3702A78D1E580232A781F43CDE576
:103CA0002A786B1C2A2A01D100F02FFC1100002475
:103CB000303918001D000294092900D9BFE50024FD
:103CC000A3001B195B005C1803001A780130110077
:103CD000303905000929F3D90294B0E501232A7887
:103CE0001F43ABE510ABDB78002B00D0E8E52023C9
:103CF00010AAD3702A78A1E50899D34A08C9069377
:103D00000023079302331F4311AB1A80CF4BB946F0
:103D10000C93089102232EE6BB0600D5BEE2FB06FB
:103D200000D55CE37B0600D5AEE3BB0500D456E3CB
:103D3000089A059908CA1970089260E52A786C2AD1
:103D400000D13FE310231F4378E5B946012B00D192
:103D5000E0E53EAC022B00D10BE10723B246A846BA
:103D60009C46069A079B5E07D7086146D8083E43E3
:103D700003003000114025003031013C3200217039
:103D80001843F0D1069207934A462F0056464546FF
:103D9000D20700D443E1302900D140E13022013C78
:103DA000BB1E22703EAAD21A4F461C000392C5E5E4
:103DB00001230398159416901490139315AE0836AA
:103DC000ABE64A46049B9B1A9A46002B00DC86E62B
:103DD000102B00DC85E39E4BA04631005446624622
:103DE000BA465F46AB461D0005E0961C1A00083136
:103DF000103C102C1ADD102310304B60531C0D604A
:103E000014901393072BF0DD002800D191E03900C6
:103E1000019812AAFFF76AFC002800D0A9E1139AC2
:103E2000103C1498561C15A9102CE4DC2B00B44649
:103E30005D460E00BB465746A2464446984643465A
:103E40003360534673606346504414901393072BBA
:103E500000DCFEE1002800D1DAE25946019812AAFE
:103E6000FFF744FC00285BD1139B039A9C46591C26
:103E7000029B14989B1A9A4615AE002B00DC35E67F
:103E8000102B00DCBDE2724BA04631005446624666
:103E9000BA465F46AB461D0005E0961C1A00083185
:103EA000103C102C19DD102310304B60531C0D609A
:103EB00014901393072BF0DD002825D039000198CA
:103EC00012AAFFF713FC002800D052E1139A103C0D
:103ED0001498561C15A9102CE5DC32002B000E009E
:103EE0005D461100BB465746A246444698464346A7
:103EF000336053465044736014901391072900DDDA
:103F000043E108360131F1E50126002215A9C7E792
:103F10005946019812AAFFF7E9FB002800D110E6E4
:103F2000DA4653465B6EDB0700D41FE653469B8997
:103F300022E60126002215A95AE7002800D153E104
:103F40005946019812AAFFF7D1FB0028E8D1139B2C
:103F500014989C46591C15AEA0E511AB159302238D
:103F600001210220169315AE8C4663460836591C73
:103F7000B1E50F20069A079BA846B4460C9E0100A7
:103F80001140715C1D071709013C3D43217019095F
:103F90000B0029002A001943F1D1069207933EAB8A
:103FA0001B1B664645464F460393C7E480234A469B
:103FB000DB0000271A404B46AA46B1463D00069E4C
:103FC000079F90463EAC03930AE00A22002330008C
:103FD0003900FCF72FFA002F00D115E206000F0080
:103FE0000A22002330003900FCF724FA4346013C42
:103FF000303222700135002BE7D00B9B1B78AB428F
:10400000E3D1FF2DE1D0002F00D0A1E1092E00D98E
:104010009EE1039B0696079755464E4699463EAB52
:104020001B1B4F46039389E41498102B00DC40E2DD
:10403000A446084B4446BA4632005F46E046AB46CB
:1040400013991D000EE0C04630780000CC640000DB
:1040500064660000546600008E1C19000832103C93
:10406000102C18DD1023103053604B1C1560149079
:104070001393072BF0DD002826D03900019812AAEF
:10408000FFF734FB002874D11399103C14984E1C90
:1040900015AA102CE6DC43462900A04634005D46F4
:1040A000A446BB46160057461C008A46534633605A
:1040B000434673606346404414901393072B00DD1E
:1040C000B1E00836591CD7E40021012615AAC6E73D
:1040D00013907B074FD54A46049B9C1A002C4ADD5F
:1040E00015AE102C00DCEBE1D74BA8461D00019B60
:1040F000102731009A46139A05E0961C1A000831E1
:10410000103C102C18DD1030531C0D604F601490C3
:104110001393072BF1DD002827D05946504612AAE9
:10412000FFF7E4FA002800D0FAE6139A103C14983E
:10413000561C15A9102CE6DC3300AA460E00454695
:1041400019005346001918C614901391072900DC72
:10415000EBE400280FD05946019812AAFFF7C6FADF
:10416000002800D0DCE61498DFE40126002215A91F
:10417000C6E7BA46F5E4049B4B4500DA4B46059A80
:1041800094469C4463460593DBE4002800D10FE687
:104190005946019812AAFFF7A9FA002800D0BFE6F5
:1041A000139B14980293591C15AE9FE4139215AEFD
:1041B00026E4029B002B01D0FFF7B4FB00233EACAA
:1041C00002930393FFF7BAFB4B46DB065DD44B46E5
:1041D0005B0656D5089A08CA9BB20693002308923C
:1041E00007930133FFF7C7FB0A9B002B70D011AB7D
:1041F000159302231693013B9C46022015AEB4E6AC
:10420000002301219C4615AE65E40699079A002417
:104210004B429441069307942D2310AAD370B946BC
:104220002C3BFFF7ABFB002800D184E059460198F6
:1042300012AAFFF75BFA002800D071E6139B1498CE
:104240009C46591C15AEFFF717FC2A780893FFF718
:10425000F5FA0836591C42E4BB0500D5EBE0089B93
:1042600004CB0692002208930792FFF780FBBB0560
:1042700000D5F5E008CA0693DB1707930892FFF70D
:1042800037FB4B469B0500D5F2E0089B04CB06921A
:104290000022089307920123FFF76DFB0899059A06
:1042A00008C91A60D2175A600891FFF7A8FA0B9B49
:1042B000002B01D1FFF704FB0B9B1B78002B01D1D6
:1042C000FFF7FEFA8023DB002A781F43FFF7B6FAD8
:1042D0009C46012115AEFFF7FEFB5C4B0C93BB0621
:1042E0004DD5072308990731994318C906930794B8
:1042F0000891FB070AD50698079903000B4305D0E0
:10430000302111AB19705A7002231F43504B1F40CC
:10431000B9460223FFF72FFBB946A3E44D4B0C939C
:10432000DDE7200001F000FD4346089300230390E1
:104330000293FFF703FB10ABDB78002B71D10A9BD4
:10434000002B00D009E69C46012115AEFFF7C7FB04
:104350000E9B0D99E41A1A00200001F013FD0B9931
:1043600030004B788C465A1E93419C4463460A2287
:104370000B9339000023FCF75DF800252EE6FB06C1
:104380000BD47B0607D5089908C99BB20693002376
:1043900008910793ADE7BB056ED4089B02CB06914D
:1043A000002108930791A4E75346986D00F014FE8E
:1043B00053469B89FFF7E0FBB946012B00D0C8E4C8
:1043C000FFF7B0FA20236A781F430135FFF736FA6A
:1043D00080239B006A781F430135FFF72FFA089A64
:1043E000059908CA19600892FFF709FA029B03931E
:1043F000062B13D8039B184C994643460893FFF7A6
:1044000020FB164B984672E5092E00D9E6E500E63A
:10441000002301219C4615AEFFF761FB06230393A1
:10442000E8E710AB03331593012301210120169314
:1044300015AEFFF730FB089A08CADBB206930023DB
:1044400008920793FFF793FA54660000B8640000DF
:10445000FFFBFFFFCC640000E06400006466000026
:1044600008CA5BB20693DB1707930892FFF740FA7E
:10447000089A08CADBB2B0E6089908C9DBB206930D
:1044800000230891079334E7089A059908CA198010
:104490000892FFF7B4F95346986D00F09DFDFFF7C1
:1044A000F2F943460893029B039300230293FFF71C
:1044B00045FA139B0F9301339C461A4B9A46F5E538
:1044C000139B0293591C174B9A463AE6594601989A
:1044D00012AAFFF70BF9002801D1FFF740FBFFF705
:1044E00040FB114B8C469846A9E45B6EDB0707D472
:1044F00053469B899B0503D45346986D00F06CFD91
:1045000001235B420593FFF73BFB089904C9029224
:10451000002A02DA0122524202926A7808911D00B2
:10452000FFF78CF95466000064660000F0B51F00C8
:1045300002231F4C1500A5440C0089896A46994343
:104540006B469981636E80211993E3890600D381BC
:10455000E369C9000793636A16A809931AAB00932D
:104560000493002302910591069300F02FFD2A0089
:104570003B0069463000FFF7FDF8051E0EDA6B467A
:104580009B895B0603D54022A3891343A381169818
:1045900000F01EFD2800074B9D44F0BD6946300029
:1045A00000F01CF90028EAD001256D42E7E7C0467B
:1045B00094FBFFFF6C040000334B70B505001868D6
:1045C0000C00002802D0836B002B3DD00C23E25E50
:1045D000A38919070DD52169002915D0D80724D53D
:1045E0000020A06060694042A0610020002924D022
:1045F00070BDD90640D55B0729D4216908231A4329
:10460000A28193B20029E9D1A02080268000B600C3
:104610001840B042E2D02100280000F00FFD0C232A
:10462000E25EA3892169D807DAD400209D0700D46F
:104630006069A06000200029DAD11B06D8D540238C
:104640001A43A2810138D3E700F02EF9BEE7216BAF
:1046500000290AD023004033994204D0280000F0FA
:104660002BFA0C23E25E0023236324239A430023C6
:10467000216963602160C1E709232B604023012089
:104680001A43A2814042B3E708032020062010B558
:1046900001F0D8FA012001F06DFDC046F0B5C64624
:1046A0000C0000B5A28980460C23C95E13074CD4C8
:1046B000802362681B010B43A381002A66DDA66A82
:1046C000002E3ED042464146156800220A609AB24A
:1046D000DB0460D4012300224046E169B047431C5B
:1046E00068D0A289A66A530706D56368C01A236BEF
:1046F000002B01D0E36BC01A00230200E1694046A1
:10470000B047431C49D143461B68002B45D01D2BA5
:1047100001D0162B57D1A3892F4A1340A381002320
:104720006360236923604346216B1D60002908D024
:1047300023004033994202D0404600F0BDF90023E7
:104740002363002004BC9046F0BD2669002EF8D0FB
:10475000236826609D1B0023920700D16369A36034
:10476000002D04DCEDE736182D1A002DE9DD2B00B5
:1047700032004046E169676AB8470028F3DC40220E
:104780000120A38940421343A381DBE7E26B002AA7
:1047900000DD94E7D5E7206DA5E7A3890E4A134015
:1047A0000022626022691BB2A3812260DB04BAD5B9
:1047B0002065B8E743461B68002B00D191E71D2B0D
:1047C00006D0162B04D04022A3891343A381B9E756
:1047D000434600201D60B5E7FFF7FFFF70B50500F9
:1047E0000C00002802D0836B002B15D00C22A35E96
:1047F000002B17D0626ED20701D49B0514D5280078
:104800002100FFF74BFF636E0500DB0702D4A3898D
:104810009B0515D5280070BD00F046F80C22A35E5C
:10482000002BE7D10025F5E7A06D00F0D3FB2800B1
:104830002100FFF733FF636E0500DB07EAD4E6E7EC
:10484000A06D00F0C9FBE5E7002310B5040003608C
:1048500043608360818143660021C2810361082235
:10486000436183615C3000F09DFF2000064BE461F2
:104870002362064B58306362054BA362054BE3622B
:1048800000F0A4FB10BDC046895C0000B15C0000D4
:10489000F15C00001D5D000010B5024900F066FBF0
:1048A00010BDC046615F000070B50400144D2800C3
:1048B00000F090FBA36B002B1DD1124A0421E26390
:1048C000B8229200A350B92303229B00E250083380
:1048D000E218043BE25060680022FFF7B5FF0122B6
:1048E0000921A068FFF7B0FF02221221E068FFF75C
:1048F000ABFF0123A363280000F06EFB70BDC04630
:10490000F83120209948000010B5024800F062FB01
:1049100010BDC0460C32202010B5024800F05CFBF0
:1049200010BDC0460C322020F0B5CE46474680B5BB
:1049300083B080468946140000F03CFB012803D177
:104940004B46013BFE2B30D9230001AF4A463900CC
:1049500040465C3301F0B0FA0600431C2BD000281F
:1049600021D03978002507E023685A1C226019708D
:104970000135B54217D2795DA368013BA360002BD6
:10498000F2DAA269934201DB0A29EDD12200404606
:1049900001F02EFA431CEBD10600300003B00CBC32
:1049A00090469946F0BD4E46F7E74B4601AFD9B267
:1049B00001263970D6E74022A3891343A381ECE78F
:1049C000536E70B505000E001400DB071ED4A189DC
:1049D0000C23D25E8B0516D580239B01194204D18E
:1049E0001A43A281626E13436366280022003100DD
:1049F000FFF79AFF636E0500DB0702D4A3899B05CE
:104A000008D5280070BDA06D00F0E4FA0C23E25E2A
:104A1000A189E1E7A06D00F0DFFAF2E7F8B50C003C
:104A2000050000F013FF204FBB685E6803239E4320
:104A30001E4B341B9C466444240B013C113324035D
:104A40009C4207DB0021280001F0BCF8BB689B19E1
:104A5000984204D0280000F001FF0020F8BD280093
:104A6000614201F0AFF8431C0DD00122BB68361B38
:104A700016435E600E4B28001A68141B1C6000F081
:104A8000EDFE0120EAE70021280001F09BF8BA685A
:104A9000831A0F2BDEDD07490968401A04490860B4
:104AA00001210B435360D5E7A4082020EF0F00003D
:104AB000B80F2020AC0C2020F0B5C64605000C0035
:104AC00000B500294FD000F0C1FE210008394C6824
:104AD000012622000320B2438F187B68834362487B
:104AE00098468368BB426BD043467B6026421ED10A
:104AF00008239C460C688444091B12198C68644581
:104B00004FD0CB68E3609C604346FC186468344235
:104B100011D1BB68554C4244A34200D17FE0FC68F0
:104B2000DC60A360012313434B608A5006E0FC184D
:104B300064683442EDD016434E603A6080239B0097
:104B40009A4213D25409D3080122A2404468DB00E0
:104B50002243426018188368C8608B608160D96006
:104B6000280000F07BFE04BC9046F0BD530A042BE5
:104B70003FD89409260039343836E40004192368F4
:104B8000083C03279C4243D05868B843904202D95E
:104B90009B689C42F8D1DC68CC608B60A160D960D6
:104BA000DEE74346F8184068304258D11300B86831
:104BB000FA6843441E43C26090604E60CB50CFE71A
:104BC00013004344264206D10A68891A8C689B1850
:104BD000CA68E260946001221A434A60244A8160F4
:104BE00012689A42BCD8234B28001968FFF716FFB9
:104BF000B6E7142B07D9542B1AD8140B26006F34A0
:104C00006E36E400BAE71E005C335B36DC00B5E7C5
:104C10000122B610B240466832434260BCE7D96018
:104C20009960CB608B60012313434B608A5097E7F8
:104C3000AA246400A34205D8D40B26007834773622
:104C4000E4009BE70C4CA34205D8940C26007D346D
:104C50007C36E40092E7FE247E26A4008EE7330033
:104C600013434B603A607BE7A4082020AC08202067
:104C7000B00C2020E80F202054050000F0B5454678
:104C8000DE4657464E46E0B5936883B00C0090462A
:104C90000090002B23D08B891A0728D50A69002A97
:104CA00025D0424616689A072DD50027AB4B002524
:104CB0009946BA46002D5AD02B004D4500D9A74B36
:104CC0005246E1690098676AB847002861DD4346AB
:104CD0009B6882442D1A181A43469860EAD1002036
:104CE00003B03CBC90469946A246AB46F0BD2100BD
:104CF0000098FFF761FC002800D02CE14246A38910
:104D000016689A07D1D4DA074BD400229146802244
:104D1000920000279346002F24D05A46A5681342DC
:104D200000D186E0AA46BD4200D9B5E09022D2006B
:104D3000134200D0C7E020685246494600F0D6FC36
:104D4000A3685D1BA5603D000027236853442360D2
:104D500043469B68A9445D1B43469D60BFD0A38921
:104D6000002FDAD13268776891460836D3E7336886
:104D700075689A4608369DE759462A0000F0B6FC49
:104D8000236821005B1900982360FFF727FD0028A6
:104D900027D00C22A35E402201201343A38140426E
:104DA0009EE7002300279A4600209B46B146002F2D
:104DB00028D0002830D05646BE4200D93E00206898
:104DC00022696369904203D9A2689D18AE42D3DC80
:104DD000B3426CDC656A5A46E1690098A847051E33
:104DE000D7DD53465B1B9A460120002B58D0434623
:104DF0009B68AB447F1B5D1B43469D6000D16EE703
:104E0000002FD6D14B461B689B464B465F68082354
:104E10009C46E144002FF5D03A000A21584600F0A4
:104E20002BFC002800D18DE05B460130C31A9A4666
:104E3000C1E720682369984216D863699A46BB4245
:104E400012D8474B38009F4200D946485146FBF7DD
:104E500007FA5346656A43434A46E1690098A84702
:104E6000051E96DD7F1B73E7BD4200D93D002A0079
:104E7000494600F03BFCA36822685B1B5219A36003
:104E80002260002BEED121000098FFF7A7FC00283C
:104E900000D07EE77F1B5BE73D00BA4620684BE70A
:104EA00021000098FFF79AFC0028A0D071E732009B
:104EB000594600F01BFCA36835009B1BA3602368C8
:104EC0009B1923608DE7606922682169551A4200A9
:104ED0001218D00F8218681C5210C0199246019502
:104EE000904201D9824602005B051AD51100009854
:104EF00000F0ECF8051E28D0019A2169FEF7A4FB0A
:104F0000A389194A134080221343A3815246019B6F
:104F10002561E818D31A3D00BA4620606261A3609B
:104F20000AE7009800F0A2FC051EEFD1009D216960
:104F30002800FFF7C1FD8022A3899343743A1BB276
:104F40002A6028E77E1CB24636E70C23009A1360DD
:104F50000C22A35E1FE701204042C1E600FCFF7F58
:104F6000FEFFFF7FFFFFFF7F7FFBFFFFF8B5474698
:104F7000CE4680B5B827804689460026BF00474404
:104F80007B68BC685D1E0DD4A389012B07D90E2256
:104F9000A35E013303D021004046C847064368346E
:104FA000013DF1D23F68002FEAD130000CBC9046A1
:104FB0009946F8BD9423024A5B00D05C7047C04616
:104FC0003807202000487047280820207047C04636
:104FD0007047C0467047C0467047C04670B50C0069
:104FE0001E000E23C95E150096B0002915DB6A4627
:104FF00001F024F8002810DBF022019B120213407C
:105000000D4A8020944663445A42534133608023C2
:10501000DB002B60000116B070BD00233360A38954
:105020001B0603D5402300202B60F4E78023DB0020
:1050300000202B60EFE7C04600E0FFFF70B58B89D2
:1050400005000C0082B09B0707D523004333236083
:1050500023610123636102B070BD6A4601ABFFF7B3
:10506000BDFF00990600280000F030F8002810D09D
:105070008022154BEB63A38920601343009A1BB277
:105080006261019AA3812061002A0CD13343A3817C
:10509000E1E70C22A35E9A05DDD4032293430222AA
:1050A0001343A381D1E728000E23E15E00F0DAFF6D
:1050B000002802D10C22A35EE8E70323A2899A43C9
:1050C000012313431BB2E1E799480000F0B54E46B7
:1050D0004546DE465746E0B50D000B35060083B069
:1050E000162D22D8102900D9B2E000F0AFFB102510
:1050F00002201823CB4FFB181A005C68083A944230
:1051000000D1B5E0032362689A431300E268A16806
:10511000CA6091600122E318596830000A435A605E
:1051200000F09CFB2000083095E007239D4300D54C
:105130008EE0A94200D98BE000F088FBFC235B00E5
:105140009D4200D2A5E1680A00D18BE0042800D975
:1051500078E138239846A80980443930C100B14F1E
:1051600079184C680839A1420ED003239C4604E00C
:10517000002ACBDAE468A14206D062466368934312
:105180005A1B0F2AF4DD40463A003C69083294422B
:1051900000D178E003236168994389460B00491BDD
:1051A0000F2900DD79E17A613A610029B2DA8022C3
:1051B0009200914500D30EE15909DA0801238B4092
:1051C000D2007968D2190B4391687B60E260A160DC
:1051D0009460CC60012182109140994259D80B42D1
:1051E00005D103229043490004300B42FBD0032336
:1051F0009846C3009946B944CC4682466346DC686B
:10520000A44507D12AE1002A00DB33E1E468A44584
:1052100000D123E14246636893435A1B0F2AF2DD13
:1052200001208046611905436560A068E56808377C
:10523000C560A86040461043F960B9604860CF601F
:1052400030008F60E25000F009FB2000083002E0DF
:105250000C230020336003B03CBC90469946A24624
:10526000AB46F0BD80213F2340209846890076E779
:10527000DC680230A34200D044E73A003C690832BF
:10528000944200D086E701217B68821091409942C8
:10529000A5D90323BC6862689A439146954203D816
:1052A000531B0F2B00DD88E023004B445E4A019323
:1052B0005E4B93461B681268EB18013200D13BE14C
:1052C0005B4A944663441B0B1B0300933000009918
:1052D00000F078FC03008046013300D1F8E0019B28
:1052E000834200D9F2E0534B19009A460968009BAB
:1052F0008C46514663440B6001991A00814200D1EB
:1053000050E15B461B68013300D155E143460199EA
:105310005B1A9A1853461A600723424641461A40C0
:105320000192194200D111E108239846881A424B94
:105330000099804441449B1A5B1A1B051B0D009188
:10534000300019009B4600F03DFC431C00D14FE1AA
:105350004346C01A03005B440093534652461B6801
:1053600001215B44136042464046BA60009A0A43FA
:105370004260BC4200D123E14A460F2A00D821E115
:1053800007200C3A824360680140052011436160A8
:10539000A118486088600F2A00D934E1424644468B
:1053A000526826490868984200D20B602449086870
:1053B000984200D38EE00B608CE001222900134359
:1053C0001143651961603000BD606B6000F046FA02
:1053D000200008303FE75A0A042A71D9142A00D95C
:1053E000C4E011005C325B31D20008235B429C4672
:1053F000BA18944463469A6803239846944500D1AA
:105400009DE0434651689943494502D992689445C5
:10541000F7D1D3689C467B686146A260E1608C60EE
:10542000D460D7E6A4082020AC0C2020E80F202070
:105430000F100000B80F202008100000E00F2020FF
:10544000E40F2020142852D9542800D996E06E2366
:105450009846280B80446F30C10080E608239B46A5
:10546000073BDC449B46DA4443465246134200D095
:10547000C4E64CE00122E318596830000A435A6040
:10548000E368A268D3609A6000F0E8F92000083071
:10549000E1E62B00E80808332CE6012360191D43E0
:1054A000656078613861C26082601A004B460A43C9
:1054B00042603000E15000F0D1F920000830CAE627
:1054C0009A09110039323831D2008EE7BC4260D0DF
:1054D000BC68626803239A43531B954202D80F2B82
:1054E00000DD6AE7300000F0B9F90020B3E65B2385
:1054F000984680445C30C10031E608235B429C46FC
:10550000E1444B469B6801384B4500D098E0434648
:105510000342F2D17B688B437B604900994200D9FA
:10552000B7E6002904D1B4E6042294464900E244D7
:105530000B42F9D050465CE610330093C6E6891062
:10554000023B8B4079680B437B6065E7009B300032
:1055500043445B421B051B0D19009B4600F032FBC8
:10556000431C00D0F4E600239B46F6E6542A2BD8D1
:105570001A0B11006F326E31D20036E7AA235B009E
:1055800098422BD8DD3B9846E80B80447830C10028
:10559000E5E52C4B009A9A461B689C4653466244AC
:1055A0001A60AEE6090500D0ABE6009ABC684A4432
:1055B00001310A436260F4E65B4642461A60ABE69C
:1055C0004446EEE641608DE7AA2149008A4224D88C
:1055D000DA0B110078327731D20006E71A4B984285
:1055E00024D87C239846A80C80447D30C100B6E5C1
:1055F000009A019B94464246083B63449B1A0093E1
:1056000000239B46A9E6210030000831FFF754FA39
:105610005346BC681B686268C3E60B498A420BD8D4
:105620009A0C11007D327C31D200DEE6FE217E2311
:105630007F209846890092E5FE227E219200D4E6E2
:105640007B686AE7B80F20205405000082B000296B
:105650000AD0002A0BD0002B0BD013780B601078E7
:10566000431E984102B0704701A9002AF3D10020DF
:10567000F8E702204042F5E770B5CCB283070DD0C1
:10568000531E002A0FD0032504E00130284206D023
:10569000013B08D30278A242F7D170BD1300032B5F
:1056A0000CD8002B01D10020F7E7C31802E001302D
:1056B0008342F8D00278A242F9D1EEE7FF220D062C
:1056C0002D0C114029430D04064E0D430268064976
:1056D0006A40511891433142E7D1043B0430032B17
:1056E000F4D8DEE780808080FFFEFEFEF0B5C6467F
:1056F00000B588420CD98B18984209D2531E002A53
:1057000003D0CA5CC254013BFBD204BC9046F0BD3E
:105710000F2A0BD80500561E002AF6D00023CC5CB9
:105720001A00EC5401339642F9D1EEE703270D003D
:105730003E0005430C0003002E402F422CD11500E3
:10574000103D2D09AC462D01A846804425681F0058
:105750001D6065685D60A5689D60E5681034DD606A
:1057600010334745F2D165460F230C2401352D0136
:10577000491913404519144211D08C59AC510436C3
:105780009C1B032CF9D80324043B9B0801339B008A
:10579000ED18C9182240BEE70500561EBEE71A00E4
:1057A000B9E7C046F0B5050083074AD0541E002A69
:1057B00044D003000322CEB202E00135013C3DD3C8
:1057C00001332E701342F8D1032C2FD9FF220A4047
:1057D000150215432A0415430F2C35D92700103F15
:1057E0003F093E01B4461E001A001036664415609B
:1057F00055609560D5601032B242F8D10F260C2268
:1058000001373F012640DB193700224217D03E1FE7
:10581000B608B400A4461A001C1D644420C2A2426B
:10582000FCD103240136B6009B193C40002C05D066
:10583000C9B21C19197001339C42FBD1F0BD340070
:10584000F4E714000300BFE72700E0E710B50248C3
:10585000FFF7C0FB10BDC046FC31202010B5024848
:10586000FFF7BAFB10BDC046FC312020F0B557460B
:105870004546DE464E46E0B50C000700904683B034
:10588000002900D1CBE045460B35FFF7DFFF162D91
:1058900070D810251023A84570D82600083E7168DE
:1058A00003220800904381460096984200DB99E06D
:1058B000C34A3018934692689446824200D1C4E0AD
:1058C000426801900092012292465046009A82431B
:1058D000019894468346DC44624650465268024230
:1058E00000D092E00320009ACB4682439446E344E2
:1058F0009B4500DB1AE152460A420FD10321326870
:10590000B21A924652688A436146511849448B46FE
:1059100099423FDA4A4493469A4240DA4146380077
:10592000FFF7D4FB8046002820D07368B44600936C
:1059300001230099020099430B00083A6344934203
:1059400000D1FAE04A46043A242A00D9FAE00300DA
:10595000132A00D9C5E02200116819605168596006
:1059600092689A6021003800FFF7A6F83800FFF728
:1059700075FF07E007239D432B1E8CDA0C233B6049
:1059800000239846404603B03CBC90469946A24648
:10599000AB46F0BD019AD3689268D3609A605346D3
:1059A0005246DB6892685646D3609A604A46043A8B
:1059B0000836242A00D99EE03300132A09D9534619
:1059C000216899606168D9601B2A00D9C8E0083451
:1059D00010332268D9461A6062685A60A26834009F
:1059E00056469A604B465B1B0F2B1DD80122494639
:1059F000736813400B4373604E4473681A437260BC
:105A00003800FFF72BFFA046BCE7084200D085E72F
:105A100003213268B21A924652688A437AE711002B
:105A2000FFF754FB8046ADE7012072687119024010
:105A30000343154375604B604E4473680831184347
:105A400070603800FFF738F8DAE7624650680322E2
:105A500090430D3282469446CA44AC44E24552DA41
:105A6000CA0700D55AE73168721A03219246526874
:105A70008A4310180100494400918C4500DD49E734
:105A800053465246DB689268D3609A6008234A46C0
:105A90005344043A9846242A7CD8132A08D95346FA
:105AA000216899606168D9601B2A78D8083410335E
:105AB00022681A6062685A60A2689A60534659194F
:105AC0005B469960009B38005A1B01231A434A60C9
:105AD0005246526813401D4353465D60FFF7BEFEB9
:105AE00050E721680160616841601B2A2ED82200BE
:105AF0000833083230E7210030003400FFF7F6FDAC
:105B0000D94656466EE75B460098A0464119996013
:105B100053465A1B01231A434A6041680B401D43F8
:105B2000456038000091FFF799FE2BE7019AD946AE
:105B3000D3689268D3609A6054E703225B6893430A
:105B400099444FE72100FFF7D1FD0BE7A168816081
:105B5000E168C160242A0CD0220010331032FBE629
:105B6000A1681961E1685961242A0BD010341833F7
:105B70002FE72269010002612200606918321833A0
:105B80004861E9E622699A61524661692033D16130
:105B900018341EE721001800FFF7A8FD8EE7A16862
:105BA0001961E1685961242A02D0103418337FE763
:105BB00022699A61524661692033D161183477E7CE
:105BC000A4082020002370B5064D040008002B60B7
:105BD00000F0BAFA431C00D070BD2B68002BFBD03C
:105BE0002360F9E71032202070B505000C001F2952
:105BF00022D8B7239B00C358002B0ED08A009B18D5
:105C00001A68002A09D0012A14D0511C0ED0002194
:105C1000200019609047002070BD280000F030F887
:105C200022000100280000F017F8F5E716230360B2
:105C30000120F1E70020EFE7162303600120404236
:105C4000EAE7C04610B5034B01001868FFF7CCFF28
:105C500010BDC04608032020002370B5074D040086
:105C6000080011002B6000F057FA431C00D070BDF3
:105C70002B68002BFBD02360F9E7C04610322020B0
:105C800010B500F039FA10BD70B50C000E25495F53
:105C900000F00EFA002803DB236D1B18236570BD8E
:105CA000A389024A1340A381F9E7C046FFEFFFFF33
:105CB000F8B50C001F000C23C95E05001600CB05CB
:105CC0000AD40A4B320019402800A1810E23E15E5C
:105CD0003B0000F01FF9F8BD0E23E15E0022022315
:105CE00000F0D2F90C23E15EEBE7C046FFEFFFFFC7
:105CF00070B50C000E25495F00F0C6F9431C06D0B4
:105D00008023A2895B011343A381206570BDA38911
:105D1000014A1340A381F9E7FFEFFFFF10B50E23FF
:105D2000C95E00F00BF910BD10B583070AD003005F
:105D3000032102E001330B4205D01A78002AF9D181
:105D4000181A10BD030019680C4A0D4C8A188A43B2
:105D500022420FD15968094A04338A188A432242E1
:105D600008D15968054A04338A188A432242F1D07F
:105D700000E001331A78002AFBD1E1E7FFFEFEFEC6
:105D800080808080F0B50C00044303000600A40767
:105D900012D1032A10D9144CA44666460D68134C40
:105DA0001F002C19AC4334421CD10433043A1E00AA
:105DB00004313D60032AF0D80024B71806E00D5DD9
:105DC000013A3555BB1A0134002D02D0002AF6D114
:105DD000F0BD0021D418002AFAD0197001339C427A
:105DE000FBD1F5E71E00E7E780808080FFFEFEFE26
:105DF000F8B505000E001400002802D0836B002BBC
:105E00004BD0A369A289A3600C23E05E13071FD5C2
:105E10002369002B1CD0FF21F7B20E40802189019D
:105E20000A4226D022686169D31A99422CDD0133D7
:105E3000A1680139A160511C2160177062699A4202
:105E40002ED0A389DB0701D50A2E29D03000F8BD5A
:105E500021002800FEF7B0FB002827D1FF21F7B270
:105E60000E408021A28989010C23E05E23690A4249
:105E7000D8D101430F4AA181616E0A40626661690F
:105E80002268D31A9942D2DC21002800FEF7A6FC32
:105E900000280BD101232268CAE7FEF705FDB0E711
:105EA00021002800FEF79AFC0028CFD00126764278
:105EB000CCE7C046FFDFFFFF70B504001D0084B0D3
:105EC000002909D0E0230B48C6582B002000B0471A
:105ED000431C0AD004B070BDE023064A01A9D6587D
:105EE0002B000022B047431CF4D100232B608A33DF
:105EF0002360EFE738072020002909D0FF2A02D8C5
:105F000001200A7070478A23036001204042F9E7AC
:105F10000020F7E770B50400080011001A00002304
:105F2000054D2B6000F01EF9431C00D070BD2B689E
:105F3000002BFBD02360F9E710322020002370B53E
:105F4000064D040008002B6000F0C6F8431C00D08A
:105F500070BD2B68002BFBD02360F9E710322020A6
:105F6000F8B506000C1E4DD0002802D0836B002B24
:105F70004AD00127636E3B4235D00C22A35E002B32
:105F800040D021003000FEF789FBE36A0500002BBA
:105F900004D03000E169984700283CDBA3891B0648
:105FA0003ED4216B002908D023004033994202D00F
:105FB0003000FEF781FD00232363616C002904D0CB
:105FC0003000FEF779FD00236364FEF79DFC00239B
:105FD000A381636EDB072CD5A06DFEF7F9FFFEF7FA
:105FE0009BFC2800F8BDA3899B05CAD4A06DFEF7D1
:105FF000F1FF0C22A35E002BC3D1636E1D003D4058
:106000003B4212D00025ECE70127FEF74DFC636E02
:106010003B42B2D1E7E70125A3896D421B06C0D5FB
:1060200030002169FEF748FDBBE7A06DFEF7D4FF05
:10603000D7E7A06DFEF7D0FFCEE7C046002370B5CE
:10604000074D0400080011002B6000F04DF8431CC0
:1060500000D070BD2B68002BFBD02360F9E7C04651
:1060600010322020002370B5064D040008002B607C
:1060700000F04AF8431C00D070BD2B68002BFBD009
:106080002360F9E71032202070B5040008001100E9
:106090001A000023054D2B6000F046F8431C00D089
:1060A00070BD2B68002BFBD02360F9E71032202055
:1060B00070B50400080011001A000023054D2B6084
:1060C00000F03AF8431C00D070BD2B68002BFBD0C9
:1060D0002360F9E71032202058220120014B404272
:1060E0001A6070471032202058220120014B404294
:1060F0001A6070471032202058220120014B404284
:106100001A607047103220205822024B00201A607B
:106110007047C0461032202058220120014B4042D7
:106120001A6070471032202058220120014B404253
:106130001A6070471032202058220120014B404243
:106140001A60704710322020044A030010680028AB
:1061500002D0C318136070470148FAE7EC0F202003
:106160001832202058220120014B40421A6070470B
:1061700010322020FEE7C04601B40248844601BC2C
:08618000604700BF0100202070
:1061880080B584B000AF78607A6888235B0101210C
:10619800D1507B68094A9B5807221340FB60FB6873
:1061A800DBB2032B03D0FB68DBB2012BF1D1FB6818
:1061B800DBB21800BD4604B080BDC046D013000055
:1061C80000000000010000000200000003000000C1
:1061D80004000000050000000600000007000000A1
:1061E800080000000C00000010000000140000006F
:1061F80018000000200000003000000040000000EF
:106208000400000005000000060000000700000070
:10621800080000000A0000000E0000001200000044
:106228003808000048080000580800006808000006
:1062380078080000AC0800009A0800008A080000EE
:106248001011121315141700564543424D53000000
:106258004D43414E203D3D2043414E4644300000D1
:106268002E2E2F4D43414C2F4D63616C5F5372634B
:106278002F697665635F6D63616C5F6D63616E2E18
:106288006300000042415544203D3D2042415544B1
:106298005F353030207C7C2042415544203D3D20F4
:1062A800424155445F32353000000000625F4D4383
:1062B800414E5F496E6974466C6167203D3D2030F0
:1062C80000000000625F4D43414E5F496E697446AD
:1062D8006C616720213D2030000000004279746520
:1062E80073203C3D20380000784D43414C5F4D43BE
:1062F800414E496E69740000784D43414C5F4D43EF
:10630800414E4465496E697400000000784D434170
:106318004C5F4D43414E547800000000784D434196
:106328004C5F4D43414E5278506F6C6C696E6700FC
:1063380000000000F8070000100000000100000045
:106348000200000048160000B415000042160000C4
:10635800BA150000FC15000002160000081600001F
:106368000E1600001416000048160000481600001B
:10637800481600004816000048160000481600009D
:10638800481600001A1600004816000048160000BB
:10639800481600004816000048160000481600007D
:1063A8004816000020160000481600004816000095
:1063B800481600004816000048160000481600005D
:1063C800481600002616000048160000481600006F
:1063D800481600004816000048160000481600003D
:1063E800481600002A16000048160000481600004B
:1063F800481600004816000048160000481600001D
:106408004816000030160000481600004816000024
:1064180048160000481600004816000048160000FC
:1064280048160000361600004816000048160000FE
:1064380048160000481600004816000048160000DC
:10644800481600003C160000010000000000000093
:106458000000000000000000200000001000000004
:106468000001000003000000000000002C00C441EF
:106478002C2066756E6374696F6E3A200000000008
:10648800617373657274696F6E20222573222066AA
:1064980061696C65643A2066696C652022257322FF
:1064A8002C206C696E65202564257325730A00000D
:1064B8003031323334353637383941424344454632
:1064C80000000000303132333435363738396162F4
:1064D8006364656600000000286E756C6C29000016
:1064E800E43C00002C3A00002C3A0000DC3C0000A0
:1064F8002C3A00002C3A00002C3A00009638000094
:106508002C3A00002C3A0000423C00008E3C00006F
:106518002C3A0000563C0000A03C00002C3A000039
:10652800983C0000903B0000903B0000903B00002E
:10653800903B0000903B0000903B0000903B000027
:10654800903B0000903B00002C3A00002C3A0000E1
:106558002C3A00002C3A00002C3A00002C3A00009B
:106568002C3A00002C3A00002C3A00002A3C00008B
:10657800CC3800002C3A00002C3A00002C3A0000DD
:106588002C3A00002C3A00002C3A00002C3A00006B
:106598002C3A00002C3A00002C3A00005439000034
:1065A8002C3A00002C3A00002C3A0000F03B000086
:1065B8002C3A00005E3C00002C3A00002C3A000007
:1065C800DA4200002C3A00002C3A00002C3A000075
:1065D8002C3A00002C3A00002C3A00002C3A00001B
:1065E8002C3A00002C3A00002C3A00002A3C00000B
:1065F800D03800002C3A00002C3A00002C3A000059
:10660800803C0000D0380000C43800002C3A00005C
:106618003C3D00002C3A0000183D000058390000AD
:10662800F83C0000C43800002C3A0000F03B0000A1
:10663800C0380000184300002C3A00002C3A000033
:106648001C4300002C3A0000C03800002020202005
:1066580020202020202020202020202030303030F2
:10666800303030303030303030303030430000009F
:10667800504F5349580000002E00000000202020F1
:1066880020202020202028282828282020202020DA
:1066980020202020202020202020202020881010AA
:1066A8001010101010101010101010101004040406
:1066B80004040404040404101010101010104141C4
:1066C80041414141010101010101010101010101B2
:1066D80001010101010101011010101010104242C6
:1066E8004242424202020202020202020202020282
:1066F8000202020202020202101010102000000022
:106708000000000000000000000000000000000081
:106718000000000000000000000000000000000071
:106728000000000000000000000000000000000061
:106738000000000000000000000000000000000051
:106748000000000000000000000000000000000041
:106758000000000000000000000000000000000031
:106768000000000000000000000000000000000021
:106778000000000000000000000000000000000011
:08678800EC9CFF7F0100000002
:10679000A10D000000000000E50E0000A90D0000A2
:1067A0008D0E0000E1080000B90B0000950B000001
:1067B000B50A0000290A0000DD0900000000000001
:1067C000000000002109000000000000000000009F
:1067D00000000000000000000000000000000000B9
:1067E0000000000000000000FF00000000000000AA
:1067F0001101000000000000000000000000000087
:106800000000000000000000000000000000000088
:106810000000000000000000000000000000000078
:106820000000000000000000000000000000000068
:106830000000000000000000000000000000000058
:106840000000000000000000000000000000000048
:106850000000000000000000000000000000000038
:106860000000000000000000000000000000000028
:106870000000000000000000008000000000020096
:1068800000800100010000000D1000001110000048
:10689000F10F000000000000000000005110000097
:1068A00000000000891000000080000001000000CE
:1068B000000000008A000000130000001300000028
:1068C00000000000000000000000000000000000C8
:1068D0000000000029000000040000000400000087
:1068E00000000000000000000000000000000000A8
:1068F00000000000000000000F0000000000000089
:1069000000000000FFFF0000000000000100000088
:106910000100000003000000030000000000000070
:106920000000000000000000000000000000000067
:106930000000000000000000000000000100000056
:10694000FF0000000A000000060000000100000037
:106950000000000002000000300000000000000005
:106960000A0000000A0000000A0000000000000009
:1069700000000000800200000A000000000000008B
:10698000AA0000004000000000000000000000001D
:10699000BE0000000A0000000A0000000100000024
:1069A000D000000000000000000000000000000017
:1069B00000000000000000000000000000000000D7
:1069C00008000000010000000100000001000000BC
:1069D000AA0000000000000000000000000000000D
:1069E00000000000000000000000000000000000A7
:1069F0000000000000000000000000000000000097
:106A00000000000000000000000000000000000086
:106A10000000000000000000000000000000000076
:106A20000000000000000000000000000000000066
:106A30000000000000000000000000000000000056
:106A40000000000000000000000000000000000046
:106A500000000000010000001003202000000000E2
:106A600000000000FC05202064062020CC06202029
:106A70000000000000000000000000000000000016
:106A80000000000000000000000000000000000006
:106A900000000000000000000000000000000000F6
:106AA00000000000000000000000000000000000E6
:106AB00000000000000000000000000000000000D6
:106AC00000000000000000000000000000000000C6
:106AD00000000000000000000000000000000000B6
:106AE00000000000000000000000000000000000A6
:106AF0000000000000000000000000000000000096
:106B00000000000000000000010000000000000084
:106B10000E33CDAB34126DE6ECDE05000B00000049
:106B20000000000000000000000000000000000065
:106B30000000000000000000000000000000000055
:106B40000000000000000000000000000000000045
:106B50000000000000000000000000000000000035
:106E800000000000000000004300000000000000BF
:106E900000000000000000000000000000000000F2
:106EA000000000000000000043000000000000009F
:106EB00000000000000000000000000000000000D2
:106EC000000000000000000043000000000000007F
:106ED00000000000000000000000000000000000B2
:106EE000000000000000000043000000000000005F
:106EF0000000000000000000000000000000000092
:106F0000000000000000000043000000000000003E
:106F10000000000000000000000000000000000071
:106F2000000000000000000043000000000000001E
:106F30000000000000000000000000000000000051
:106F400000000000000000004300000000000000FE
:106F50000000000000000000000000000000000031
:106F60000000000000000000F95E00004D56000027
:106F70000000000084660000806600008464000059
:106F80008464000084640000846400008464000061
:106F90008464000084640000846400008464000051
:106FA000FFFFFFFFFFFFFFFFFFFFFFFFFFFF0000EF
:106FB0000100415343494900000000000000000067
:106FC00000000000000000000000000000000000C1
:106FD0000000415343494900000000000000000048
:106FE00000000000000000000000000000000000A1
:106FF000000000000000000000000000A4082020A5
:10700000A4082020AC082020AC082020B4082020B0
:10701000B4082020BC082020BC082020C408202060
:10702000C4082020CC082020CC082020D408202010
:10703000D4082020DC082020DC082020E4082020C0
:10704000E4082020EC082020EC082020F408202070
:10705000F4082020FC082020FC082020040920201F
:10706000040920200C0920200C09202014092020CC
:10707000140920201C0920201C092020240920207C
:10708000240920202C0920202C092020340920202C
:10709000340920203C0920203C09202044092020DC
:1070A000440920204C0920204C092020540920208C
:1070B000540920205C0920205C092020640920203C
:1070C000640920206C0920206C09202074092020EC
:1070D000740920207C0920207C092020840920209C
:1070E000840920208C0920208C092020940920204C
:1070F000940920209C0920209C092020A4092020FC
:10710000A4092020AC092020AC092020B4092020AB
:10711000B4092020BC092020BC092020C40920205B
:10712000C4092020CC092020CC092020D40920200B
:10713000D4092020DC092020DC092020E4092020BB
:10714000E4092020EC092020EC092020F40920206B
:10715000F4092020FC092020FC092020040A20201A
:10716000040A20200C0A20200C0A2020140A2020C7
:10717000140A20201C0A20201C0A2020240A202077
:10718000240A20202C0A20202C0A2020340A202027
:10719000340A20203C0A20203C0A2020440A2020D7
:1071A000440A20204C0A20204C0A2020540A202087
:1071B000540A20205C0A20205C0A2020640A202037
:1071C000640A20206C0A20206C0A2020740A2020E7
:1071D000740A20207C0A20207C0A2020840A202097
:1071E000840A20208C0A20208C0A2020940A202047
:1071F000940A20209C0A20209C0A2020A40A2020F7
:10720000A40A2020AC0A2020AC0A2020B40A2020A6
:10721000B40A2020BC0A2020BC0A2020C40A202056
:10722000C40A2020CC0A2020CC0A2020D40A202006
:10723000D40A2020DC0A2020DC0A2020E40A2020B6
:10724000E40A2020EC0A2020EC0A2020F40A202066
:10725000F40A2020FC0A2020FC0A2020040B202015
:10726000040B20200C0B20200C0B2020140B2020C2
:10727000140B20201C0B20201C0B2020240B202072
:10728000240B20202C0B20202C0B2020340B202022
:10729000340B20203C0B20203C0B2020440B2020D2
:1072A000440B20204C0B20204C0B2020540B202082
:1072B000540B20205C0B20205C0B2020640B202032
:1072C000640B20206C0B20206C0B2020740B2020E2
:1072D000740B20207C0B20207C0B2020840B202092
:1072E000840B20208C0B20208C0B2020940B202042
:1072F000940B20209C0B20209C0B2020A40B2020F2
:10730000A40B2020AC0B2020AC0B2020B40B2020A1
:10731000B40B2020BC0B2020BC0B2020C40B202051
:10732000C40B2020CC0B2020CC0B2020D40B202001
:10733000D40B2020DC0B2020DC0B2020E40B2020B1
:10734000E40B2020EC0B2020EC0B2020F40B202061
:10735000F40B2020FC0B2020FC0B2020040C202010
:10736000040C20200C0C20200C0C2020140C2020BD
:10737000140C20201C0C20201C0C2020240C20206D
:10738000240C20202C0C20202C0C2020340C20201D
:10739000340C20203C0C20203C0C2020440C2020CD
:1073A000440C20204C0C20204C0C2020540C20207D
:1073B000540C20205C0C20205C0C2020640C20202D
:1073C000640C20206C0C20206C0C2020740C2020DD
:1073D000740C20207C0C20207C0C2020840C20208D
:1073E000840C20208C0C20208C0C2020940C20203D
:1073F000940C20209C0C20209C0C2020FFFFFFFFE1
:08740000000002000000000082
:040000030000800079
:00000001FF
